:106DB6000000050200000301FA0400EF0500030AC3
:106DC6000A5A0B001E0C00FA0D00030E00040F01F8
:106DD60064100096120132130AFA14010217010A0E
:106DE6001801EF1905321A010A1B01EF1C05321FA3
:106DF600FFFF20FFFF23011E2400642A00FA2B0058
:106E0600FA2C50782D003D2E004630006432507822
:106E16003300003432FF35016436016437015038DF
:106E26000A643A00033B00043C00643E003C3F0019
:106E36000140FFFF411450420A5A430AC844053232
:106E46004500B44600FA4900024B00014C00FA50D6
:106E56000606510596520A32530B46540A965705B2
:106E660046590A465A32FA5B010A5C0A325E000A41
:106E76005F00646200FE64021C67FFFF680101692F
:106E860001016A05966B00006C32FF6D0004730009
:106E9600007400007801327901327E00648100645A
:106EA60084FFFF8800028A00019D0A969E00019FCA
:106EB600FFFFA0013CA2000AA3FFFFA40064A500F7
:106EC60064A6FFFFA7FFFFA8FFFFA9FFFF01013C84
:106ED6001500022F003C4701784802045602024E74
:106EE600FFFF58000261FFFF6600028500AF8600C3
:106EF600018700FA890108990006A100FAFAFAFA50
:106F060001013C1500022F1E3C4701784802045639
:106F160002024EFFFF58000261FFFF660002850075
:106F2600AF8600018700FA890108990000A10000D8
:106F3600FAFAFA0065006F00790083008D00970069
:106F4600A100AC00B600C000CA00D400DE00E80014
:106F5600F200580060006800700078008000880029
:106F660090009800A000A800B000B800C100C800BA
:106F7600D000D800DF00E600EE00F6004100470032
:106F86004D00530059005F0065006C0071007700EA
:106F96007D00830089008F0095009B00A200A7005A
:106FA600AC00B200B900C000C500CA00D200D500CE
:076FB600DD00E100E700EF40
:103D750075A71085F97385FA747E017F00E57412C5
:103D850070CFE5732FFF50010E8E598F5A90001892
:103D9500E0FCA3E0FDEF2DFDEE3CFC8C5B8D5C9023
:103DA5000038E0FAA3E0FBED2BFBEC3AFA8A5B8BDB
:103DB5005C2275A71085F97385FA747E017F00E58D
:103DC500741270CFE5732FFF50010E8E598F5AACC8
:103DD5002CAD2DEF2DFDEE3CFC8C5B8D5C90003801
:103DE500E0FAA3E0FBED2BFBEC3AFA8A5B8B5C2255
:103DF500E55CF5FBE55BF5FCD29322E55CF5E9E5D1
:103E05005BF5EAD29422E55CF5EBE55BF5ECD29146
:103E150022E55CF5EDE55BF5EED29222E55CF5FD7C
:103E2500E55BF5FED28722E55CF5CEE55BF5CFD205
:103E35009022A203B34004D2978002C29722E50CD8
:103E45009069A5F8282873806CA237B34008E5B5BA
:103E55004408F5B58006E5B554F7F5B58057A237A2
:103E6500B34008E5B54402F5B58006E5B554FDF562
:103E7500B58042A2379297803CA237B34008E5B59A
:103E85004410F5B58006E5B554EFF5B58027A237A2
:103E9500B34008E5B54420F5B58006E5B554DFF532
:103EA500B58012A2379292800CA23792878006A223
:053EB50037929080002F
:1069A500023E4C023E4E023E63023E78023E7E02AD
:0E69B5003E93023EA8023EAE023EB4023EBA3F
:103EBA0022743690015EF0743090015FF0742D9098
:103ECA000160F07432900161F07420900162F07424
:103EDA0042900163F0744D900164F074579001654B
:103EEA00F07420900166F0744D900167F07433907D
:103EFA000168F07420900169F0744590016AF074C9
:103F0A003490016BF0743690016CF022900895E0C1
:103F1A00FEA3E0FF741DD39F74019E400C906DB602
:103F2A00120048E493F599802E90F802E493B405C0
:103F3A0014900895E0FEA3E0FF906DE9120048E4B2
:103F4A0093F5998012900895E0FEA3E0FF906DB674
:103F5A00120048E493F5999008951270DD9008953F
:103F6A00E0FEA3E0FFEFB45007EEB40103754D0085
:103F7A0022AE59AF5A74068E048F05FF1270BF8C99
:103F8A005B8D5CAE59AF5A74068E048F05FF1270B2
:103F9A00EA8C598D5AE55A455960137406C3955AE5
:103FAA00FFE49559FE8E598F5A785B127122E57398
:103FBA00A85BB80015D3955C4010E573C3955CFF08
:103FCA00E4955BFE8E5B8F5C8010E573243CC395A1
:103FDA005CFFE4955BFE8E5B8F5CAE5BAF5C743B13
:103FEA006F4E6006743C6F4E701AAE5BAF5C743BEA
:103FFA006F4E70057573018003757302755C3A75AF
:10400A005B0080037573002290009BE0B40104C238
:10401A00078002D20790009CE0B40104C208800223
:10402A00D2089000D9E075F0D2A4FFAEF0740A8EDF
:10403A00048F05FF1270BF900889ECF0A3EDF09091
:10404A0000D9E075F02BA4FFAEF0900014EEF0A3B7
:10405A00EFF07E017F00900097E01270CF9000DAB7
:10406A00E08E048F05FF1270BF740AFF1270BF8DB5
:10407A00609000E3E075F0D2A4FFAEF0740A8E04FB
:10408A008F05FF1270BF90088DECF0A3EDF0900041
:10409A00E5E060139000E5E0F5F0741684FF7E0019
:1040AA00EF9008EBF0800674649008EBF09000DB68
:1040BA00E0900076F0900127E0900082F0900129CC
:1040CA00E0FE9000D7E08E0088F0A4FFAEF0EF90FB
:1040DA0008F4F0900102E075F013A4FDACF0900032
:1040EA0038ECF0A3EDF0A220B34016900173E07013
:1040FA000C900174E07006900175E060028002C2C3
:10410A0020900173E0B4300F900174E0B447089036
:10411A000175E0643B60028004D2218002C22190D2
:10412A000094E0FE9008F5E06E601B7599E61201B6
:10413A009C74AB900050F01206DA7464F5097508A5
:10414A000012062480FE90008CE070067400900035
:10415A00C1F090007AE0FE9000C1E0B506579000E9
:10416A007CE0FE9000DFE0B5064B90007BE0FE901D
:10417A0000EDE0B5063F900080E0FE900094E0B5C7
:10418A00063390007DE0FE9000CFE0B50627900050
:10419A007EE0FE9000FAE0B5061B90007FE0FE90FC
:1041AA0000FBE0B5060F900081E0FE90010DE06E85
:1041BA00700302439990009CE070089000DDE0646F
:1041CA00046002800674039000DDF09000CFE0D313
:1041DA00940250069000EDE060087405900110F01A
:1041EA0080067408900110F0900094E0B4010674FF
:1041FA0000900094F0900094E0B4020674009000DD
:10420A00DFF0900094E0B4030674009000ECF090A4
:10421A00010DE06014742A900785F074009006D1AD
:10422A00F074009006D2F0800C7400900785F07448
:10423A002A9006D1F09000DFE0D39401401A741856
:10424A00900112F07400900113F074009006D5F0FA
:10425A0074009006D6F0803D9000EDE0B40108901D
:10426A0000CFE064036002801A7400900112F074B7
:10427A0018900113F074009006D5F074009006D6D9
:10428A00F080127400900112F07400900113F0741F
:10429A00189006D5F09000C1E0601474079000A849
:1042AA00F074009006D9F074009006DAF0800C746D
:1042BA00009000A8F074079006D9F09000C1E0B40D
:1042CA00021474089000A9F074009006DDF07400DE
:1042DA009006DEF0800C74009000A9F07408900635
:1042EA00DDF09000CFE0B402069000EDE0600280BD
:1042FA002674049006E1F074059006E5F0740690C1
:10430A0006E9F07400900780F07400900781F07459
:10431A0000900782F0803674009006E1F0740090F5
:10432A0006E2F074009006E5F074009006E6F07478
:10433A00009006E9F074009006EAF0740490078091
:10434A00F07405900781F07406900782F0D21F90EE
:10435A0000C1E090007AF09000EDE090007BF090D0
:10436A0000DFE090007CF09000CFE090007DF090BC
:10437A000094E0900080F09000FAE090007EF090C7
:10438A0000FBE090007FF090010DE0900081F0903A
:10439A0000F7E0B40117900024740FF0A374FFF043
:1043AA00900026E4F0A3F074029000F7F09000F772
:1043BA00E0B40341900026E0FEA3E0FF900024E071
:1043CA00FCA3E0FD12711A74101270CF7408120067
:1043DA0039EF9000F6F0EF700674FF9000F6F07473
:1043EA00009000F7F0900025E09000ADF0900024D6
:1043FA00E09000AEF0900088E0900085F090008791
:10440A00E0900084F09000B6E0C3941E50569000ED
:10441A00B6E0F404241E900086F0900086E075F061
:10442A000684FF7E008F73900086E075F00684ADE7
:10443A00F07C008D74900084E0D39574400D900058
:10444A0084E0C39574900084F0800F900084E02487
:10445A0006C39574900084F00573900085E0257377
:10446A00900085F0900085E0900046F0900046E0CC
:10447A002414900047F0900046E02428900048F069
:10448A00900047E0D3943C400B900047E0C3943C33
:10449A00900047F0900048E0D3943C400B900048CD
:1044AA00E0C3943C900048F090004CE4F090004641
:1044BA00E0643B6007900046E0B43C20900046E090
:1044CA00B43B06740290004CF0900046E0B43C06FF
:1044DA0090004C7401F09000467401F090004DE495
:1044EA00F0900047E0643B6007900047E0B43C204E
:1044FA00900047E0B43B06740290004DF0900047EC
:10450A00E0B43C0690004D7401F09000477401F04D
:10451A0090004EE4F0900048E0643B600790004849
:10452A00E0B43C20900048E0B43B06740290004E90
:10453A00F0900048E0B43C0690004E7401F0900000
:10454A00487401F0900088E0FE9000EBE02E9000A5
:10455A0051F0900051E0D3943C400B900051E0C3DD
:10456A00943C900051F0900051E0D3943C400B9061
:10457A000051E0C3943C900051F09000C6E0B401B1
:10458A0063900051E0641E6007900051E0B43C065D
:10459A00900051E004F0900051E0641D6007900023
:1045AA0051E0B43B06900051E014F0900051E0D382
:1045BA00943C400B900051E0C3943C900051F09021
:1045CA000051E0D3941E400D900051E0C3941E9018
:1045DA000052F0800A900051E0241E900052F075BB
:1045EA005D1E8079900051E06414600F900051E0E4
:1045FA0064286007900051E0B43C06900051E00442
:10460A00F0900051E06413600F900051E06427605D
:10461A0007900051E0B43B06900051E014F090007E
:10462A0051E0D3943C400B900051E0C3943C90007D
:10463A0051F0900051E0D39414400B900051E0C324
:10464A009414900051F0900051E0D39414400B90D0
:10465A000051E0C39414900051F0755D14900088E5
:10466A00E0FE9000CEE0D39E5013900088E0FE90CA
:10467A0000CEE0F4042E04900049F08013900088E4
:10468A00E02478FE9000CEE0F4042E04900049F075
:10469A00900049E075F01484AFF07E00EF4E70068A
:1046AA00900049E004F0900049E00475F01484AFEA
:1046BA00F07E00EF4E7006900049E014F090004939
:1046CA00E0B479069000497401F0900049E0D3946F
:1046DA003C400F900049E0C3943C900049F0D21A44
:1046EA008002C21A900049E0241490004AF0900017
:1046FA0049E0242890004BF090004AE0D3943C40D3
:10470A000B90004AE0C3943C90004AF090004BE0C2
:10471A00D3943C400B90004BE0C3943C90004BF088
:10472A0012019C22C293C294C291C292C287C290C1
:10473A00E5B554EFF5B5E5B554DFF5B5C296C295C2
:10474A00C2A0C297C2A2C2A1E5B554BFF5B5E5B5EC
:10475A00547FF5B5E5B554FBF5B5C209755E4690CB
:10476A0000D1E07005756D028003756D0375540004
:10477A0075530090000C74FFF0A374DCF0C20FC2F2
:10478A0011C21374C890003AF074C890003EF074D5
:10479A00C8900042F0755200755100C20475460077
:1047AA00E56FB41303756F0075630090001AE4F0A7
:1047BA00A3F0757010C20CC20DC20EC2037556006A
:1047CA0075550090000EE4F0A3F0900010E4F0A3F9
:1047DA00F0C227755800755700900093E075F032C3
:1047EA00A4FFAEF0900022EEF0A3EFF0900083E475
:1047FA00F09008F1E4F0C222C218C219C21AC21B10
:10480A00900012E4F0A3F022755A00755900AE59CF
:10481A00AF5A741CC39F74019E5003024906906DDF
:10482A00B6120048E493645F6023906DB6120048A4
:10483A00E493647E6017906DB6120048E493648135
:10484A00600B906DB6120048E493B484030248E604
:10485A00AE59AF5A906DB6120048E4939000871291
:10486A0071000FBF00010EE0FC906DB6120048EC1B
:10487A00FEE493FFEEC39F5026AE59AF5A0FBF0016
:10488A00010E906DB6120048AE59AF5AE493FC90EF
:10489A006DB6120048E493900087127100ECF0AEF6
:1048AA0059AF5A906DB6120048E49390008712717E
:1048BA0000E0FC906DB8120048ECFCE493FDECD3E8
:1048CA009D4019906DB8120048E493FC906DB612A1
:1048DA000048E493900087127100ECF0AE59AF5A89
:1048EA0074022FFF50010E8E598F5A785A7401267E
:1048FA00F6500418E436F6400302481822755A00A6
:10490A00755900AE59AF5A7432BE00039F50030264
:10491A0049D4906ED3120048E49390008712710034
:10492A000FBF00010EE0FC906ED3120048ECFEE4CB
:10493A0093FFEEC39F5026AE59AF5A0FBF00010E28
:10494A00906ED3120048AE59AF5AE493FC906ED3DE
:10495A00120048E493900087127100ECF0AE59AF50
:10496A005A906ED3120048E493900087127100E0C7
:10497A00FC906ED5120048ECFCE493FDECD39D400C
:10498A0019906ED5120048E493FC906ED312004839
:10499A00E493900087127100ECF0AE59AF5A742D6F
:1049AA006F4E7006755A33755900AE59AF5A740274
:1049BA002FFF50010E8E598F5A785A740126F650DD
:1049CA000418E436F6400302490D22755A00755957
:1049DA0000AE59AF5A7432BE00039F5003024AA276
:1049EA00906F06120048E4939000871271000FBF7F
:1049FA0000010EE0FC906F06120048ECFEE493FF03
:104A0A00EEC39F5026AE59AF5A0FBF00010E906FEA
:104A1A0006120048AE59AF5AE493FC906F06120092
:104A2A0048E493900087127100ECF0AE59AF5A90A7
:104A3A006F06120048E493900087127100E0FC9020
:104A4A006F08120048ECFCE493FDECD39D401990EA
:104A5A006F08120048E493FC906F06120048E49332
:104A6A00900087127100ECF0AE59AF5A742D6F4E58
:104A7A007006755A33755900AE59AF5A74022FFF32
:104A8A0050010E8E598F5A785A740126F65004181E
:104A9A00E436F640030249DB2275A71085F97385CF
:104AAA00FA747E017F00E5741270CFE5732FFF5010
:104ABA00010E8E598F5AAC5BAD5CEF2DFDEE3CFCBE
:104ACA008C5B8D5C123DF5123E00123E0B9000CFBE
:104ADA00E0D394024009123E16123E21123E2C7572
:104AEA00A7002285F97385FA747E017F00E57412A6
:104AFA0070CFE5732FFF50010E8E598F5A7E017FBA
:104B0A007690010CE01270CFAC59AD5AED2FFFEC44
:104B1A003EFE8E5B8F5CE55CF5EDE55BF5EE9000A5
:104B2A0076E4F07412900054F02285F97385FA74D1
:104B3A007E017F00E5741270CFE5732FFF50010EDE
:104B4A008E598F5A900014E0FCA3E0FDEF2DFDEE84
:104B5A003CFC8C5B8D5CE55CF5FDE55BF5FE2205B6
:104B6A006422A2DBB340089000DBE0900076F0A25A
:104B7A00DCB34024A29650067419900054F0A29512
:104B8A0050067419900054F0A2A0500674199000AF
:104B9A0054F0C296C295C2A075D8402285A77275F4
:104BAA00A7109000CFE0D3940250079000EDE0B434
:104BBA000252A2D8B34002C293A2D9B34002C2940D
:104BCA00A2DAB34002C2919000CFE064026007907B
:104BDA0000CFE0B40417A2DBB34002C292A2DCB356
:104BEA004002C287A2DDB34002C2908015A2D8B3A8
:104BFA004002C292A2D9B34002C287A2DAB34002EB
:104C0A00C290802DA2D8B3400AC2939000EDE06012
:104C1A0002C292A2D9B3400AC2949000EDE06002A7
:104C2A00C287A2DAB3400AC2919000EDE06002C2E4
:104C3A009075D8408572A72290F800E493640660C4
:104C4A000280FE12009E75A70075D80075D90475FA
:104C5A00DD0975DE0975D84075A71075D80075D9B4
:104C6A000475DA0975DB0975DC0975DD0975DE0974
:104C7A0075DF0975D84075A7001200FB74C8F509DD
:104C8A0075080012062475A70FE5FC900063F0E58D
:104C9A00FB900064F0E5FA900065F0E5F990006693
:104CAA00F075A70090F800E493F5271207439008DF
:104CBA009EE0D39403500790089EE0B40106740066
:104CCA0090089EF090089EE09008F5F0740190001C
:104CDA00D0F090089EE09069C3F8282873802A8053
:104CEA002875A70F75F30F75A700A2A340067402D3
:104CFA009000D0F0801375A70F75F31775A700A25F
:094D0A00A4400674029000D0F0F0
:0C69C300024CE7024CE9024CEB024D00D4
:104D13009000D0E0B4022AC217120AEC7402900089
:104D2300D0F090089EE09069CFF828287380108017
:0F4D33000E74009000DFF0800674009000ECF02A
:0C69CF00024D30024D32024D34024D3CAE
:104D42008028D217120A0174019000D0F090089EB8
:104D5200E09069DBF82828738010800E74009000C0
:0A4D6200DFF0800674009000ECF012
:0C69DB00024D5A024D5C024D5E024D66FA
:104D6C0090F807E493900070F0900070E044089085
:104D7C000070F0900070E054FE900070F01203BDD3
:104D8C00123EBB9008ABE0900173F09008ACE09041
:104D9C000174F09008ADE0900175F0900173E07033
:104DAC000C900174E07006900175E060028004C202
:104DBC00208002D2209000C1E00490007AF0900193
:104DCC002BE0B4FF06740090012BF090012CE0B4A2
:104DDC00FF06740090012CF012481290F802E49334
:104DEC00B405051249D5800312490774009000F7E9
:104DFC00F0124012E5B54401F5B57406900056F07A
:104E0C007400900057F07401900058F090F802E490
:104E1C0093900059F090F803E49390005AF090F8B6
:104E2C0004E49390005BF0740690005CF0900059E1
:104E3C00E0B40506740590005CF0744690005DF0DB
:104E4C00740390005EF0740790005FF074019000A2
:104E5C0060F090F805E493900061F090F806E4930C
:104E6C00900062F0740090006AF0740090006BF097
:104E7C00740090006CF0740090006DF07400900061
:104E8C006EF0740090006FF074FF900071F0A2B699
:104E9C00B39205A2B3B39206A2A4B3921DA2A3B37C
:104EAC00921E900072E4F0756F00743A900787F0D0
:104EBC0074FD900788F0900073E4F0756E0190001B
:104ECC0054E4F09000D1E0B40106741A900054F050
:104EDC00C21C756300C20AD20BC203757100C21FDB
:104EEC001205C6755F00756B0075610075653275CE
:104EFC006600756700756800756900756A0090003A
:104F0C001AE4F0A3F0756C00D2B2D2A4D2B0D2B134
:104F1C00D2A3D2A7D2A6D2A5D2B77E017F00900091
:104F2C00AEE01270CF9000ADE02FFF50010E90005C
:104F3C0024EEF0A3EFF0EFD394FFEE940F40079024
:104F4C000024E4F0A3F09000F6E0700674FF9000EB
:104F5C00F6F09000D1E07005756D028003756D035D
:104F6C00741C900114F0741A900115F074009001E7
:104F7C0016F07400900117F074299006CDF074159A
:104F8C00900775F07416900776F07417900777F009
:104F9C007400900778F07400900779F07400900713
:104FAC007AF0740090077BF0740090077CF0740129
:104FBC0090077DF0740290077EF0740390077FF0E9
:104FCC007400900783F07400900784F0D29CE57015
:104FDC00D3941040037570109006CEE0D3940C401F
:104FEC000674009006CEF09006D2E0D3940C4006E6
:104FFC0074009006D2F09006D6E0D3940C40067460
:10500C00009006D6F09006DAE0D3940C40067400BB
:10501C009006DAF09006DEE0D3940C400674009013
:10502C0006DEF09006E2E0D3940C40067400900685
:10503C00E2F09006E6E0D3940C400674009006E68D
:10504C00F09006EAE0D3940C400674009006EAF067
:10505C00D2EC75CF01A298B34005C298120C54E55E
:10506C004D6006A299B3B340028005C2991210E0BC
:10507C00E54E64016005E54EB4040280D5C28E7E17
:10508C00107F00E5641270CFE58D75F010A4FDACB7
:10509C00F0EF2DFDEE3CFCE58B75F01084FF7E00EF
:1050AC00ED2FFFEC3EFE8E538F54D28E9000B4E069
:1050BC0060099000B4E0C3943D4002805690001CFF
:1050CC001270DD90001CE0FEA3E0FF90001EE0FCDF
:1050DC00A3E0FDEFB5053CEEB50438B215A204B360
:1050EC004013A215B34008E5B54404F5B58006E5B8
:1050FC00B554FBF5B590001EE0FEA3E0FF90002038
:10510C00E0FCA3E0FDEF2DFDEE3CFC90001EECF06E
:10511C00A3EDF09000C1E060099000C1E0C39403DE
:10512C0040028077123027A20440089000ABE0F5D3
:10513C0045801BE55FC395605005754500800F9059
:10514C000098E0C3956150069000BEE0F545E5453A
:10515C0075F002A4FFAEF0900893EEF0A3EFF0AC64
:10516C002EAD2FEDD39FEC9E4015E5B554EFF5B564
:10517C009000C1E0B40206E5B54420F5B5801C9062
:10518C000072E0C394415013E5B54410F5B590009E
:10519C00C1E0B40206E5B554DFF5B59000C1E0B44A
:1051AC000324123142AE2EAF2F900893E0FCA3E003
:1051BC00FDEFD39DEE9C4008E5B554EFF5B58006A8
:1051CC00E5B54410F5B590009CE06009A2B330063B
:1051DC0001B3B340028039A2B3300601B34031A20F
:1051EC00B3300801B3401C9000CFE0B40306A21802
:1051FC00B3B3400280067405900054F0D218A20894
:10520C00B39206A208B330B301B34004A2089206CD
:10521C00A2B6300501B350030257EBA2B63005011C
:10522C00B350030257EBA2B6300701B35003025739
:10523C0009756E009000B4E0B43D13A207B34008AA
:10524C00E5B554FBF5B58006E5B54404F5B5055E4A
:10525C00A209B3B35013AE53AF5490000CE0FCA3AF
:10526C00E0FDEDC39FEC9E40030253BCE56DB4031F
:10527C002EA227B34022E55EB43B03756D01E55EBB
:10528C00C3943B50069000547401F0E55ED3943BFC
:10529C0040067402900054F0755E01D227805CE5E4
:1052AC006DB40206756D01755E3BE55EB43B05752C
:1052BC005E018047900054E07032E55EC3943B5031
:1052CC00069000547401F0E55ED3943B40067402E2
:1052DC00900054F0E55EC3943B5002D21CE55ED3C3
:1052EC00943B4002D21CC296C295C2A09000D1E061
:1052FC00B4010512472E8003755E01AE55AF56AC56
:10530C0053AD54EF2DFDEE3CFC74028C068D071250
:10531C0000398E558F569000B4E060099000B4E0CF
:10532C00C3943D4002804390001CE0FEA3E0FF903C
:10533C0000B4E08E048F05FF1270BF74018C068DD3
:10534C0007120039900020EEF0A3EFF0900020E05F
:10535C00F8A3E090001EC8F0A3C8F090001CE4F085
:10536C00A3F0C215E5B554FBF5B5A2A4B34002C237
:10537C001DA2A3B34002C21EA21CB34002C21CA2B7
:10538C0018B34006A21A92198002B21990009CE040
:10539C006012E56D700EA218B35009A219301A01F3
:1053AC00B3B3400280067405900054F0C218803AE2
:1053BC00AE55AF56AC53AD54EF2DFDEE3CFC740125
:1053CC008C068D071200398E558F56E56DC39402ED
:1053DC00500DAC53AD5474B8C39D740B9C400280FB
:1053EC000912472E7406900054F0E55EB43B12741B
:1053FC0003900054F0D21C9000D1E0B4010312478A
:10540C002EAE57AF58AC53AD54EF2DFDEE3CFC8C8B
:10541C00578D58AE53AF54EFD39DEE9C4011900076
:10542C0012E0FAA3E0FBEBC394E8EA940340028099
:10543C00069000121270DD900010E0FEA3E0FFACAD
:10544C0053AD54EF2DFDEE3CFC900010ECF0A3EDB1
:10545C00F09000D1E0B40118AE53AF547405127043
:10546C00CF740112003990000CEEF0A3EFF0801114
:10547C00AE53AF5474021270CF90000CEEF0A3EF49
:10548C00F0C28E758D00758B0075640075540175B6
:10549C005300D28EE55E240E75F00F84AFF07E00C3
:1054AC00EF4E6003025535E56D6013AE55AF567483
:1054BC000F1270CF90000EEEF0A3EFF0800F900063
:1054CC0010E0F8A3E090000EC8F0A3C8F090000E16
:1054DC00E0FEA3E0FFEF4E600B7C7C7D1A126FBDEB
:1054EC008E518F52900010E4F0A3F0AE51AF527475
:1054FC0028BE00039F5010E5632FFF50010E74016E
:10550C001200398E518F528552639000D8E0A85109
:10551C00B8000DD395524008E552900053F0800925
:10552C009000D8E014900053F09000CFE0B4040841
:10553C00900049E0655E6002800BA219B34004D272
:10554C001B8002B21BE55E640B6005E55EB42909A5
:10555C009000C1E06003122CDD9000C6E0B4011491
:10556C00900051E0655E6007900052E0B55E0375F7
:10557C006F00801E900051E0655E6013900051E05A
:10558C002414655E6009900051E02428B55E037513
:10559C006F00A20AB35006A209B3B34003025651DE
:1055AC0090008DE0B4017390010FE0B4021412125C
:1055BC0081900077E075F0BCA4FFAEF08E5B8F5C41
:1055CC008056E56775F00A84FF7E0090058712000F
:1055DC0048E0F55A755900AE59AF5A9000B2E01236
:1055EC0070CF74648E048F05FF1270BF8C5B8D5C62
:1055FC00E55C90004FF0AE59AF5A90008BE0127002
:10560C00CF74648E048F05FF1270BF74BC8C068D32
:10561C00071270CF8E5B8F5C801790008BE075F05B
:10562C00BCA4FFAEF08E5B8F5C9000B2E090004F9C
:10563C00F0E561C394CC5006E55C455B70028003D9
:10564C00124AA3D20AE56DB40106E55E641160024C
:10565C0080097570009000557401F0E56D600302CF
:10566C0057049000D4E0600D900076E0A851B8008B
:10567C00069552400280409000D4E0B4021F900086
:10568C0046E0655E600F900047E0655E6007900045
:10569C0048E0B55E03757003756C00800CC2017533
:1056AC006C0090001AE4F0A3F0900076E0600674B1
:1056BC0009900054F08041900046E0655E600F90C8
:1056CC000047E0655E6007900048E0B55E2A7570A3
:1056DC0000900046E0B55E069000557401F0900015
:1056EC0047E0B55E067402900055F0900048E0B5B6
:1056FC005E067403900055F0A207B39205A207B39F
:10570C0030B601B350030257EB756E019000B4E054
:10571C00B43D13A207B34008E5B54404F5B58006C3
:10572C00E5B554FBF5B5E5B54401F5B5742B900022
:10573C0072F0A2079205E55ED3944A4014D209E5B3
:10574C005ED39485400B7404900054F0D21C755EAB
:10575C00469000DCE0B40107E56AC3944140028046
:10576C0018E56AC3941450087413900054F0800622
:10577C00740E900054F012472E90005CE0FE9000E6
:10578C0059E0C39E4009900059E0D3940840097435
:10579C00FB900054F012472E90005AE060159000D8
:1057AC005AE0FE900058E06E600974FC900054F0D2
:1057BC0012472E90005BE0601590005BE0FE9000BD
:1057CC005DE06E600974FE900054F012472E900854
:1057DC009EE0600690010CE060028003120BD7A2E1
:1057EC001CB34006C296C295C2A090010CE0600C9E
:1057FC00AE51AF527414BE00059F4002803790002A
:10580C0094E09069E7F8282873802A8028A2A3B333
:10581C005005A21EB340028005124AEDD21E80151F
:10582C00A2A4B35005A21DB340028005124AEDD2CA
:05583C001D8002800048
:1069E70002581502581702581902582C02583F022C
:0269F700584105
:10584100A20CB3B35008900049E0655E60030259B1
:10585100AFA202B35006A201B3B340030259A9900B
:1058610000CFE0B40402800302596D123D75900827
:10587100F1E0B40202800302595BA21BB3406790BE
:105881000120E0601F900018E0FEA3E0FF900118E6
:10589100E01270CF74C88E048F05FF1270BF8C5B4D
:1058A1008D5C800A900018E0F55BA3E0F55CAE5BCF
:1058B100AF5C745E1270CF74058E048F05FF127099
:1058C100BFAE59AF5AED2FFFEC3EFE8E5B8F5C9061
:1058D1000038E0FCA3E0FDEF2DFDEE3CFC8C5B8D80
:1058E1005C123DF58068900120E0D39403401F9045
:1058F1000018E0FEA3E0FF90011BE01270CF74C816
:105901008E048F05FF1270BF8C5B8D5C800A900046
:1059110018E0F55BA3E0F55CAE5BAF5C745E127002
:10592100CF74058E048F05FF1270BFAE59AF5AEDCB
:105931002FFFEC3EFE8E5B8F5C900038E0FCA3E015
:10594100FDEF2DFDEE3CFC8C5B8D5C123E16900054
:10595100EDE0B40103123E378010123DF5123E1600
:105961009000EDE0B40103123E378039123D75120B
:105971003DF59000CFE0B4030ED2929000EDE0B47B
:105981000103123E37801E9000EDE0B40206123D85
:10599100B7123E169000EDE0B40106A203B3B34086
:1059A100028002D29275A700C20CD20DD20EA20DB6
:1059B100B3B3500890004AE0655E6003025B30A219
:1059C10002B35006A201B3B34003025B2A9000CF99
:1059D100E0B404028003025ADE123D759008F1E042
:1059E100B402028003025ACCA21BB3406A90012088
:1059F100E0D39401401F900018E0FEA3E0FF900166
:105A010019E01270CF74C88E048F05FF1270BF8C1D
:105A11005B8D5C800A900018E0F55BA3E0F55CAE5D
:105A21005BAF5C745E1270CF74058E048F05FF123C
:105A310070BFAE59AF5AED2FFFEC3EFE8E5B8F5C0F
:105A4100900038E0FCA3E0FDEF2DFDEE3CFC8C5B0B
:105A51008D5C123E008068900120E0D39404401FC9
:105A6100900018E0FEA3E0FF90011CE01270CF74DB
:105A7100C88E048F05FF1270BF8C5B8D5C800A900D
:105A81000018E0F55BA3E0F55CAE5BAF5C745E1201
:105A910070CF74058E048F05FF1270BFAE59AF5AD7
:105AA100ED2FFFEC3EFE8E5B8F5C900038E0FCA397
:105AB100E0FDEF2DFDEE3CFC8C5B8D5C123E2190F8
:105AC10000EDE0B40103123E378010123E00123E99
:105AD100219000EDE0B40103123E378049123D757B
:105AE100123E009000EDE0C394025007A203B340C0
:105AF10002D2879000CFE0B4030ED2879000EDE090
:105B0100B40103123E37801E9000EDE0B40206128C
:105B11003DB7123E219000EDE0B40106A203B3B3FC
:105B210040028002D28775A700D20CC20DD20EA20C
:105B31000EB3B3500890004BE0655E6003025CB1A8
:105B4100A202B35006A201B3B34003025CAB9000C2
:105B5100CFE0B404028003025C5F123D759008F14E
:105B6100E0B402028003025C4DA21BB3406A9001C3
:105B710020E0D39402401F900018E0FEA3E0FF90C4
:105B8100011AE01270CF74C88E048F05FF1270BF26
:105B91008C5B8D5C800A900018E0F55BA3E0F55CFE
:105BA100AE5BAF5C745E1270CF74058E048F05FF1F
:105BB1001270BFAE59AF5AED2FFFEC3EFE8E5B8FD8
:105BC1005C900038E0FCA3E0FDEF2DFDEE3CFC8C89
:105BD1005B8D5C123E0B8068900120E0D394054000
:105BE1001F900018E0FEA3E0FF90011DE01270CFAE
:105BF10074C88E048F05FF1270BF8C5B8D5C800AA8
:105C0100900018E0F55BA3E0F55CAE5BAF5C745E01
:105C11001270CF74058E048F05FF1270BFAE59AF9D
:105C21005AED2FFFEC3EFE8E5B8F5C900038E0FC5E
:105C3100A3E0FDEF2DFDEE3CFC8C5B8D5C123E2C58
:105C41009000EDE0B40103123E378010123E0B12BA
:105C51003E2C9000EDE0B40103123E378049123D25
:105C610075123E0B9000EDE0C394025007A203B3FE
:105C71004002D2909000CFE0B4030ED2909000ED9C
:105C8100E0B40103123E37801E9000EDE0B402063D
:105C9100123DB7123E2C9000EDE0B40106A203B311
:105CA100B340028002D29075A700D20CD20DC20E71
:0D5CB100E5709069F9F82828739000F4E080
:0369F900025CBA83
:105CBE00906A2CF828287312260C801212260C805B
:0E5CCE000D12269680081227428003122742EC
:0F6A2C00025CC5025CCA025CCF025CD4025CD97A
:105CDC007570010261C212286E122985757002025C
:105CEC0061C2122D21A204B340139000D9E075F0CB
:105CFC001DA4FFAEF0900014EEF0A3EFF090088717
:105D0C00E0FEA3E0FF740A1270CF90000EE0FCA33B
:105D1C00E0FD74098F02FF1270BF8D078C038E0497
:105D2C008A058B06126FBD90088BEEF0A3EFF07412
:105D3C00F0BE00039F500B74F090088BF8E4F0E871
:105D4C00A3F0E536700375360190088BE0FEA3E0F6
:105D5C00FFE5362FFF50010E90088BEEF0A3EFF00D
:0B5D6C00757003A22E401A900055E055
:0669FC00025CE2025CEE09
:105D7700906A3BF8282873800D75700A8008757043
:065D87000B800375700C97
:0C6A3B00025D7E025D80025D85025D8AC6
:105D8D000261C29006CEE060077401F508122E4F35
:105D9D00A230B3B35008900785E0642A60028009F1
:105DAD00E5B54402F5B5025E579000C2E0D394020A
:105DBD004045900096E02403A851B8000495525038
:105DCD0009900098E0D395615002800ED202A22670
:105DDD0040067408900054F0D226900096E0A85129
:105DED00B80005D39552500B900098E02403C3954D
:105DFD00615002C2028053900096E02403A851B86E
:105E0D00000495525010E55FC395605009900098BD
:105E1D00E0D395615002800ED202A226400674088E
:105E2D00900054F0D226900096E0A851B80005D30A
:105E3D0095525014E560240FC3955F400B90009868
:105E4D00E02403C395615002C202A2024002C226A1
:105E5D00A230B3500DA202B35008900785E0642A1A
:105E6D0060028006E5B554FDF5B59000DCE07007E5
:105E7D00E56AC3941440028002D2029000D1E0B4CE
:105E8D000102D202A2024005757004800A757010DD
:0E5E9D0090001AE4F0A3F00261C29000C2E08F
:066A0200025D90025EA798
:105EAB00906A47F828287312139780121213978061
:0E5EBB000D12154A80081216018003121601FE
:0F6A4700025EB2025EB7025EBC025EC1025EC6B4
:105EC9009006D2E060077402F508122E4F7570052E
:105ED9000261C212175A7570069006D6E0600774FF
:105EE90003F508122E4F9006DAE060077404F508EE
:105EF900122E4F0261C290004FE06006A204B3B3B4
:105F09004002800DE55ED39414500690004FE014D2
:105F1900F01219E37570079006DEE060077405F565
:105F290008122E4F9006E2E060077406F508122E5B
:105F39004F0261C290010FE0B40203121308121E4E
:105F49004B7570089006E6E060077407F508122E95
:105F59004F9006EAE060077408F508122E4F0261B7
:105F6900C2121F2D7570090261C2122305A20CB35A
:105F79005005A20DB340028006D20CD20DD20E7587
:105F890070100261C290003CE0C394465008C2966A
:105F9900744690003CF090004CE0B4011DE53624B5
:105FA90006F53690088BE0FEA3E0FF74062FFF503C
:105FB900010E90088BEEF0A3EFF090004CE0B402D4
:105FC9001DE536240CF53690088BE0FEA3E0FF743E
:105FD9000C2FFF50010E90088BEEF0A3EFF08536E1
:105FE9005A755900900046E0F573123F7BE55C90C5
:105FF900003CF0900006E559F0A3E55AF0E57390EE
:10600900003DF0C21090088BE0F559A3E0F55A90D5
:106019000046E0F573123F7BE55C90003AF0900092
:1060290000E559F0A3E55AF0E57390003BF0C20F83
:10603900E56DB4010575700B80037570030261C2CB
:10604900900040E0C394465008C2957446900040C1
:10605900F090004DE0B4011DE5362406F5369008B0
:106069008BE0FEA3E0FF74062FFF50010E90088B12
:10607900EEF0A3EFF090004DE0B4021DE536240CDC
:10608900F53690088BE0FEA3E0FF740C2FFF50015A
:106099000E90088BEEF0A3EFF085365A75590090F3
:1060A9000047E0F573123F7BE55C900040F09000FB
:1060B90008E559F0A3E55AF0E573900041F0C212E2
:1060C90090088BE0F559A3E0F55A900047E0F57385
:1060D900123F7BE55C90003EF0900002E559F0A389
:1060E900E55AF0E57390003FF0C211E56DB4010582
:1060F90075700C80037570030261C2900044E0C39F
:1061090094465008C2A07446900044F090004EE0B6
:10611900B4011DE5362406F53690088BE0FEA3E0B0
:10612900FF74062FFF50010E90088BEEF0A3EFF0DD
:1061390090004EE0B4021DE536240CF53690088B2C
:10614900E0FEA3E0FF740C2FFF50010E90088BEEC8
:10615900F0A3EFF085365A755900900048E0F573C1
:10616900123F7BE55C900044F090000AE559F0A3EA
:10617900E55AF0E573900045F0C21490088BE0F5FC
:1061890059A3E0F55A900048E0F573123F7BE55CAE
:10619900900042F0900004E559F0A3E55AF0E57348
:1061A900900043F0C213E56DB40103756D0075707D
:0961B900038006800480028000CE
:106A0800025EDC025EFF025F3D025F6A025F7302A4
:106A18005F8E0260490261040261BC0261BE0261CC
:046A2800C00261C285
:1061C20090003AE0B55E028003026264A20F407260
:1061D200900000E0FEA3E0FFEF4E6021AE55AF5607
:1061E200900000E0FCA3E0FD12000374068E048F11
:1061F20005FF1270BF900000ECF0A3EDF090003BA1
:10620200E0601A900000E0FEA3E0FFAC55AD56EF4F
:106212002DFDEE3CFC900000ECF0A3EDF090003B75
:10622200E0D39401401A900000E0FEA3E0FFAC55D9
:10623200AD56EF2DFDEE3CFC900000ECF0A3EDF02E
:10624200D20FAE53AF54900000E0FCA3E0FDEFC3C9
:106252009DEE9C400D124B34D296C20F74C8900032
:106262003AF0A20FB3B3500790003AE0B55E028055
:106272000D124B34D29674C890003AF0C20F9000BF
:106282003CE0B55E02800302631FA21040729000E0
:1062920006E0FEA3E0FFEF4E6021AE55AF56900040
:1062A20006E0FCA3E0FD12000374068E048F05FFD6
:1062B2001270BF900006ECF0A3EDF090003DE0609C
:1062C2001A900006E0FEA3E0FFAC55AD56EF2DFD9F
:1062D200EE3CFC900006ECF0A3EDF090003DE0D324
:1062E2009401401A900006E0FEA3E0FFAC55AD56C3
:1062F200EF2DFDEE3CFC900006ECF0A3EDF0D21089
:10630200AE53AF54900006E0FCA3E0FDEFC39DEE58
:106312009C400AC296744690003CF0C210A210B390
:10632200B3500790003CE0B55E02800AC296744604
:1063320090003CF0C21090003EE0B55E0280030285
:1063420063DAA2114072900002E0FEA3E0FFEF4E7A
:106352006021AE55AF56900002E0FCA3E0FD1200B2
:106362000374068E048F05FF1270BF900002ECF0DA
:10637200A3EDF090003FE0601A900002E0FEA3E07F
:10638200FFAC55AD56EF2DFDEE3CFC900002ECF05B
:10639200A3EDF090003FE0D39401401A900002E098
:1063A200FEA3E0FFAC55AD56EF2DFDEE3CFC900098
:1063B20002ECF0A3EDF0D211AE53AF54900002E024
:1063C200FCA3E0FDEFC39DEE9C400D124B34D29531
:1063D200C21174C890003EF0A211B3B350079000EE
:1063E2003EE0B55E02800D124B34D29574C8900027
:1063F2003EF0C211900040E0B55E02800302649557
:10640200A2124072900008E0FEA3E0FFEF4E60216E
:10641200AE55AF56900008E0FCA3E0FD12000374F5
:10642200068E048F05FF1270BF900008ECF0A3EDFA
:10643200F0900041E0601A900008E0FEA3E0FFAC9B
:1064420055AD56EF2DFDEE3CFC900008ECF0A3EDAF
:10645200F0900041E0D39401401A900008E0FEA3BE
:10646200E0FFAC55AD56EF2DFDEE3CFC900008EC84
:10647200F0A3EDF0D212AE53AF54900008E0FCA3AB
:10648200E0FDEFC39DEE9C400AC295744690004029
:10649200F0C212A212B3B35007900040E0B55E0200
:1064A200800AC2957446900040F0C212900042E009
:1064B200B55E028003026550A2134072900004E0B0
:1064C200FEA3E0FFEF4E6021AE55AF56900004E010
:1064D200FCA3E0FD12000374068E048F05FF127008
:1064E200BF900004ECF0A3EDF0900043E0601A903E
:1064F2000004E0FEA3E0FFAC55AD56EF2DFDEE3CEF
:10650200FC900004ECF0A3EDF0900043E0D3940182
:10651200401A900004E0FEA3E0FFAC55AD56EF2D0B
:10652200FDEE3CFC900004ECF0A3EDF0D213AE5370
:10653200AF54900004E0FCA3E0FDEFC39DEE9C404D
:106542000D124B34D2A0C21374C8900042F0A213B1
:10655200B3B35007900042E0B55E02800D124B3497
:10656200D2A074C8900042F0C213900044E0B55E1D
:1065720002800302660BA214407290000AE0FEA39E
:10658200E0FFEF4E6021AE55AF5690000AE0FCA34B
:10659200E0FD12000374068E048F05FF1270BF9097
:1065A200000AECF0A3EDF0900045E0601A90000ABA
:1065B200E0FEA3E0FFAC55AD56EF2DFDEE3CFC90A6
:1065C200000AECF0A3EDF0900045E0D39401401AEC
:1065D20090000AE0FEA3E0FFAC55AD56EF2DFDEEB4
:1065E2003CFC90000AECF0A3EDF0D214AE53AF5491
:1065F20090000AE0FCA3E0FDEFC39DEE9C400AC2BE
:10660200A07446900044F0C214A214B3B350079091
:106612000044E0B55E02800AC2A07446900044F0D5
:10662200C2149000DFE0B4020280030267409000CF
:1066320074E0D395665064900074E0F4042566FE1D
:106642009000E2E08E00F5F0E884FF7E008F73EFA9
:10665200C39410500CEF8573F0A4FDACF08D7380E1
:10666200037573FF900074E0D39573400B90007430
:10667200E0C39573F57180037571009000FDE0D35E
:10668200957140069000FDE0F5719000FEE0C39523
:106692007150069000FEE0F5718071900074E0C3C5
:1066A2009566FE9000E2E08E00F5F0E884FF7E0041
:1066B2008F73EFC39410500CEF8573F0A4FDACF010
:1066C2008D7380037573FF85735A7559009000743A
:1066D200E0255AFFAE5950010E8E598F5A74FFBEF3
:1066E2000009D39F4005855A7180037571FF9000A0
:1066F200FDE0D3957140069000FDE0F5719000FE3B
:10670200E0C3957150069000FEE0F571A204B3B3A8
:10671200500D900075E0FE9000EAE0D39E5002809A
:106722000A7407900054F0C297801375A710E5CD44
:10673200C395714004C2978002D29775A700A20444
:10674200B35003026804900104E0A851B800049514
:10675200525017900103E0A851B8000ED395524051
:1067620009900105E0D395614002802375A710E5E9
:10677200CDC394805008E5B54480F5B58006E5B5F3
:10678200547FF5B5E5B554BFF5B575A70080217501
:10679200A710E5CDC394805008E5B54440F5B58017
:1067A20006E5B554BFF5B5E5B5547FF5B575A70057
:1067B200900107E0A851B8000495525017900106C5
:1067C200E0A851B8000ED395524009900108E0D3D9
:1067D20095614002801775A710E5CDC394805004DF
:1067E200D2A18002C2A1C2A275A700801575A7100E
:1067F200E5CDC394805004D2A28002C2A2C2A17588
:10680200A700E56FC39413501DE56F75F00284AFC6
:10681200F07E00EF4E70051232FC800AA2EDB3400A
:1068220005C2ED1232FCAE53AF547410C39F7427ED
:106832009E400C900073E0C3945A40030269A2A2E6
:1068420009B3400912472E7406900054F0A20BB30C
:10685200500EE561D394334007E561C394CC400206
:10686200804190010FE0B40214121281900077E08F
:1068720075F05EA4FFAEF08E5B8F5C800F90008B94
:10688200E075F05EA4FFAEF08E5B8F5CE55C455B6D
:106892006011E5B54401F5B5742B900072F0124A0F
:1068A200A3D20B900073E0D394014007E561C39437
:1068B2001A40028002C20B9006CEE060077401F516
:1068C20008122E4F9006D2E060077402F508122ECD
:1068D2004F9006D6E060077403F508122E4F90061B
:1068E200DAE060077404F508122E4F9006DEE060CD
:1068F200077405F508122E4F9006E2E06007740651
:10690200F508122E4F9006E6E060077407F50812AC
:106912002E4F9006EAE060077408F508122E4F9099
:106922000073E0C3945A5010E56FB41309900073DA
:10693200E004F0756F00803FE56FB41303756F00DC
:10694200C28E758D00758B00756400755401755388
:1069520000D28E900072E0C394415008900072E021
:1069620004F080067441900072F0900072E0B4412D
:1069720006E5B554FEF5B5900073E0D394014007E7
:10698200E56AC3944140028006740E900054F09070
:10699200089EE0600690010CE060028003120BD7B3
:0369A20002505E42
:106A56000000010001400160018001A001C001E0C9
:106A660002000300039603B603D603F404000500F0
:106A76000512052405360548055A056C057E059060
:106A860005A805C005DE0600061406280646066E9D
:106A960006AE05CF06EE00FF013F015F017F019FB5
:106AA60001BF01DF01FF02FF039503B503D503F321
:106AB60003FF04FF05110523053505470559056B39
:106AC600057D058F05A705BF05CE05F1061306272B
:106AD6000645066D06AD06ED05DD06FF0FAA0FA5F8
:106AE6000F9F0F9A0F940F8D0F870F800F780F71DE
:106AF6000F680F600F570F4E0F450F3B0F300F25D6
:106B06000F1A0F0E0F020EF50EE80EDB0ECC0EBEA0
:106B16000EAE0E9F0E8E0E7D0E6C0E5A0E470E3466
:106B26000E200E0C0DF70DE20DCB0DB50D9D0D854E
:106B36000D6D0D540D3A0D200D050CE90CCE0CB162
:106B46000C940C760C580C3A0C1B0BFB0BDB0BBB9A
:106B56000B9A0B790B570B350B130AF10ACE0AABBE
:106B66000A870A640A400A1C09F809D409B0098C84
:106B760009670943091F08FB08D608B2088E086A88
:106B86000846082307FF07DC07B90796077307516E
:106B9600072F070D06EC06CA06AA068906690649E6
:106BA600062A060A05EC05CD05B0059205750558B9
:106BB600053C0520050504EA04CF04B5049C0482BF
:106BC6000469045104390422040B03F403DE03C8E8
:106BD60003B2039D038903750361034D033B032839
:106BE6000316030402F202E102D102C002B002A0BF
:106BF600029102820273026502570249023C022F89
:106C060002220216020901FD01F201E601DB01D0B2
:106C160001C601BB01B101A7019D0194018B01824F
:106C26000179017001680160015801500148014174
:106C360001390132012B0125011E01180111010B39
:106C4600010500FF00FA0FA60FA00F990F920F8BF8
:106C56000F840F7C0F740F6B0F620F580F4E0F438C
:106C66000F380F2C0F1F0F120F050EF70EE80ED858
:106C76000EC80EB70EA50E930E800E6C0E580E4261
:106C86000E2C0E150DFD0DE40DCB0DB10D950D79E8
:106C96000D5D0D3F0D200D010CE10CC00C9E0C7C12
:106CA6000C590C350C100BEA0BC40B9E0B760B4FD4
:106CB6000B260AFD0AD40AAA0A800A550A2A09FFDF
:106CC60009D409A8097C0950092508F908CD08A1A5
:106CD6000875084A081E07F307C8079D0773074982
:106CE600072006F706CE06A6067E06570630060AD3
:106CF60005E405BF059B057705540532051004EF2D
:106D060004CE04AE048F047104530435041903FD44
:106D160003E203C703AD0394037B0363034B03340E
:106D2600031E030802F302DE02CA02B602A30291A0
:106D3600027F026D025C024C023C022C021D020E16
:106D4600020001F201E401D701CA01BE01B101A6A8
:106D5600019A018F0185017A01700166015D015377
:106D6600014A0141013901310129012101190112AB
:106D7600010B010400FD00F700F000EA00E400DE6C
:106D860000D900D300CE00C900C400BF00BA00B5C8
:106D960000B100AD00A800A400A0009C00990095D9
:106DA6000091008E008A008700840081007E007BAF
:10009E0075B50075840175A70075FFA075EF069004
:1000AE000050E4F075C91075A70F75A1C775A700AC
:1000BE0075D90075CE0C75A70F75F1FE75F2FF752B
:1000CE00F30775F47875A4BA75A5FF75A60775AE16
:1000DE000075AFFF75D48175D5FF75D6FF75D7FF47
:1000EE0075A70075A20175A14775F8092275E60876
:1000FE0075E71075BC0175BE0475BD6C75BE0775D0
:10010E00BDA075BE0875BD0175BC0075BB1875BC6C
:10011E002075BA0875E88075D11375A70F75E105BE
:10012E0075E20075C74012472E759700759780745B
:10013E000A1270AF7597C0E5975420700280F8755B
:10014E008F0275A700D2AF75980075A90C75A70F11
:10015E0075AB4375ADFB75AC1E75A71075C91875DB
:10016E00CA0075CB0075C80475A700758912758E07
:10017E0004758C00758A00C2A9D28C758D00758BA2
:10018E0000D2ABD28E75B62075D944C2992290009A
:10019E0089E090089DF0900094E090089EF0900009
:1001AE0095E090089FF09000B4E09008A0F09000C9
:1001BE00C1E09008A1F09000CFE09008A2F090006E
:1001CE00DDE09008A3F09000DFE09008A4F090002E
:1001DE00EDE09008A5F09000FAE09008A6F09000EF
:1001EE00FBE09008A7F090010DE09008A8F09001B8
:1001FE0025E09008AAF0900173E09008ABF0900112
:10020E0074E09008ACF0900175E09008ADF09001AC
:10021E000CE09008AEF09000F6E09008AFF0900081
:10022E00ADE09008B0F09000AEE09008B1F0900014
:10023E00A8E09008B2F09000A9E09008B3F0900109
:10024E0012E09008B4F0900113E09008B5F0900120
:10025E0014E09008B6F0900115E09008B7F0900108
:10026E0016E09008B8F09006CDE09008B9F0900630
:10027E00D1E09008BAF09006D5E09008BBF0900659
:10028E00D9E09008BCF09006DDE09008BDF0900635
:10029E00E1E09008BEF09006E5E09008BFF0900611
:1002AE00E9E09008C0F09006EDE09008C1F09006ED
:1002BE00F1E09008C2F0900775E09008C3F0900747
:1002CE0076E09008C4F0900777E09008C5F09007AC
:1002DE0078E09008C6F0900779E09008C7F0900794
:1002EE007AE09008C8F090077BE09008C9F090077C
:1002FE007CE09008CAF090077DE09008CBF0900764
:10030E007EE09008CCF090077FE09008CDF090074B
:10031E0080E09008CEF0900781E09008CFF0900733
:10032E0082E09008D0F0900783E09008D1F090071B
:10033E0084E09008D2F0900785E09008D3F0900109
:10034E0017E09008D4F0900118E09008D5F09001D5
:10035E0019E09008D6F090011AE09008D7F09001BD
:10036E001BE09008D8F090011CE09008D9F09001A5
:10037E001DE09008DAF090011EE09008DBF090018D
:10038E001FE09008DCF0900120E09008DDF0900076
:10039E00BBE09008DEF09000F3E09008DFF09001F3
:1003AE002BE09008E0F090012CE09008E1F0229014
:1003BE00089DE0900089F090089EE0900094F090E7
:1003CE00089FE0900095F09008A0E09000B4F090A7
:1003DE0008A1E09000C1F09008A2E09000CFF0904C
:1003EE0008A3E09000DDF09008A4E09000DFF0900C
:1003FE0008A5E09000EDF09008A6E09000FAF090CD
:10040E0008A7E09000FBF09008A8E090010DF09096
:10041E0008AAE0900125F09008AEE090010CF09053
:10042E0008AFE09000F6F09008B0E09000ADF090CC
:10043E0008B1E09000AEF09008B2E09000A8F09005
:10044E0008B3E09000A9F09008B4E0900112F0908B
:10045E0008B5E0900113F09008B6E0900114F0900A
:10046E0008B7E0900115F09008B8E0900116F090F2
:10047E0008B9E09006CDF09008BAE09006D1F09061
:10048E0008BBE09006D5F09008BCE09006D9F0903D
:10049E0008BDE09006DDF09008BEE09006E1F09019
:1004AE0008BFE09006E5F09008C0E09006E9F090F5
:1004BE0008C1E09006EDF09008C2E09006F1F090D1
:1004CE0008C3E0900775F09008C4E0900776F090AE
:1004DE0008C5E0900777F09008C6E0900778F09096
:1004EE0008C7E0900779F09008C8E090077AF0907E
:1004FE0008C9E090077BF09008CAE090077CF09066
:10050E0008CBE090077DF09008CCE090077EF0904D
:10051E0008CDE090077FF09008CEE0900780F09035
:10052E0008CFE0900781F09008D0E0900782F0901D
:10053E0008D1E0900783F09008D2E0900784F09005
:10054E0008D3E0900785F09008D4E0900117F09062
:10055E0008D5E0900118F09008D6E0900119F090BF
:10056E0008D7E090011AF09008D8E090011BF090A7
:10057E0008D9E090011CF09008DAE090011DF0908F
:10058E0008DBE090011EF09008DCE090011FF09077
:10059E0008DDE0900120F09008DEE09000BBF090C6
:1005AE0008DFE09000F3F09008E0E090012BF0906F
:1005BE0008E1E090012CF022754700900895E4F0D8
:1005CE00A3F0753100753000754D00754E00C22ACE
:1005DE00D22B90089EE06002D21F74FE900897F80E
:1005EE00E4F0E8A3F074FE90089BF8E4F0E8A3F0C2
:1005FE0074FE900899F8E4F0E8A3F0745A9008EFAE
:10060E00F0745A9008F0F0D22CC228C22EC22DC21D
:10061E0029C230C23622750B00750A00AE0AAF0B26
:10062E00AC08AD09EDC39FEC9E401674FF1270AF7F
:10063E0075CF01780B740126F6500418E436F65087
:10064E00DB22C2AF75D904758F0375B7A575B7F1E7
:10065E0090F800E4F0758F0175B7A575B7F1E52731
:10066E0090F800F075B7A575B7F190F801E4F07544
:10067E00B7A575B7F19008E3E090F802F075B7A54D
:10068E0075B7F19008E7E090F803F075B7A575B768
:10069E00F19008E4E090F804F075B7A575B7F19005
:1006AE0008E5E090F805F075B7A575B7F19008E686
:1006BE00E090F806F075B7A575B7F19008E8E090F0
:1006CE00F807F0758F0075D944D2AF22900050E034
:1006DE00B4AB61C2AF75D90475B62275F522758FAC
:1006EE000375B7A575B7F1740090F600F0758F011C
:1006FE00755A00755900AE59AF5A7445BE00279F02
:10070E00402475B7A575B7F190089D120048E0FC1E
:10071E0090F600120048ECF0785A740126F6500458
:10072E0018E436F650D0758F0075F51175B6207534
:10073E00D944D2AF22C2AF75F52275D904755A00CD
:10074E00755900AE59AF5A7445BE00229F401F9096
:10075E00F600120048E493FC90089D120048ECF05D
:10076E00785A740126F6500418E436F650D575D929
:10077E004475F511D2AF22900050E0B4AA02800366
:10078E000208C2C2AF75D90475B62275F522758FEF
:10079E000375B7A575B7F1740090F400F075B7A5A1
:1007AE0075B7F1740090F200F075B7A575B7F174D6
:1007BE000090F000F075B7A575B7F1740090EE00DB
:1007CE00F0758F01755A00755900AE59AF5A74FF06
:1007DE00C39F74019E402475B7A575B7F19000872D
:1007EE00120048E0FC90F400120048ECF0785A74C5
:1007FE000126F6500418E436F650CF755A00755996
:10080E0000AE59AF5A74FFC39F74019E402475B752
:10081E00A575B7F1900287120048E0FC90F2001225
:10082E000048ECF0785A740126F6500418E436F6B7
:10083E0050CF755A00755900AE59AF5A74FFC39F09
:10084E0074019E402475B7A575B7F1900487120008
:10085E0048E0FC90F000120048ECF0785A74012643
:10086E00F6500418E436F650CF755A00755900AE9E
:10087E0059AF5A74FFC39F74019E402475B7A57576
:10088E00B7F1900687120048E0FC90EE0012004887
:10089E00ECF0785A740126F6500418E436F650CF70
:1008AE00758F0075F51175B62075D944D2AF743AAF
:1008BE00900787F022900050E0B4AA028003020A4B
:1008CE0000C2AF75D90475B62275F522758F037502
:1008DE00B7A575B7F1740090EC00F075B7A575B7B4
:1008EE00F1740090EA00F075B7A575B7F174009039
:1008FE00E800F075B7A575B7F1740090E600F075D5
:10090E008F01755A00755900AE59AF5A74FFC39FC7
:10091E0074019E402475B7A575B7F190008712003B
:10092E0048E0FC90EC00120048ECF0785A74012676
:10093E00F6500418E436F650CF755A00755900AECD
:10094E0059AF5A74FFC39F74019E402475B7A575A5
:10095E00B7F1900287120048E0FC90EA00120048BE
:10096E00ECF0785A740126F6500418E436F650CF9F
:10097E00755A00755900AE59AF5A74FFC39F740172
:10098E009E402475B7A575B7F1900487120048E014
:10099E00FC90E800120048ECF0785A740126F650EC
:1009AE000418E436F650CF755A00755900AE59AF9B
:1009BE005A74FFC39F74019E402475B7A575B7F195
:1009CE00900687120048E0FC90E600120048ECF01A
:1009DE00785A740126F6500418E436F650CF758F07
:1009EE000075F51175B62075D944D2AF743A9007DB
:1009FE0087F022C2AF75D90475F522755A00755964
:100A0E0000AE59AF5A74FFC39F74019E401F90F4FD
:100A1E0000120048E493FC900087120048ECF07836
:100A2E005A740126F6500418E436F650D4755A005E
:100A3E00755900AE59AF5A74FFC39F74019E401F83
:100A4E0090F200120048E493FC900287120048ECEA
:100A5E00F0785A740126F6500418E436F650D47520
:100A6E005A00755900AE59AF5A74FFC39F74019E58
:100A7E00401F90F000120048E493FC90048712008F
:100A8E0048ECF0785A740126F6500418E436F65005
:100A9E00D4755A00755900AE59AF5A74FFC39F747E
:100AAE00019E401F90EE00120048E493FC900687D2
:100ABE00120048ECF0785A740126F6500418E43609
:100ACE00F650D475F51175D944D2AF74019000D09B
:100ADE00F0743A900787F09008F67401F022C2AFD6
:100AEE0075D90475F522755A00755900AE59AF5A6D
:100AFE0074FFC39F74019E401F90EC00120048E4E7
:100B0E0093FC900087120048ECF0785A740126F698
:100B1E00500418E436F650D4755A00755900AE5983
:100B2E00AF5A74FFC39F74019E401F90EA001200DB
:100B3E0048E493FC900287120048ECF0785A740156
:100B4E0026F6500418E436F650D4755A007559003E
:100B5E00AE59AF5A74FFC39F74019E401F90E800B8
:100B6E00120048E493FC900487120048ECF0785A87
:100B7E00740126F6500418E436F650D4755A0075F2
:100B8E005900AE59AF5A74FFC39F74019E401F9017
:100B9E00E600120048E493FC900687120048ECF041
:100BAE00785A740126F6500418E436F650D475F5CA
:100BBE001175D944D2AF74029000D0F0743A9007F8
:100BCE0087F074029008F6F02274019000D0F09035
:100BDE00089EE0903CBBF828287380188016A2A3CC
:100BEE00400674029000D0F0800AA2A4400674025F
:040BFE009000D0F0A3
:0C3CBB00020BE8020BEA020BEC020BF813
:100C02009000D0E0B40105A234B34002801AD2347D
:100C120012472E120A0174019000D0F01203BD1285
:100C22003EBB741B900054F09000D0E0B40206A2C8
:100C320034B3B34002801AC23412472E120AEC7443
:100C4200029000D0F01203BD123EBB741B90005400
:100C5200F022E54E64046006E59964FF600280318B
:100C6200A22A4004D22A8027E54E600874E6254E67
:100C7200900054F0E54D600874F0254D900054F05A
:100C8200E54EB4010280FE754E00754D00C22A8009
:100C920002C22AE54E903CC7F8282873754E00E53B
:100CA20099B4FF03754D01E599B4FE03754D02E554
:100CB20099B4FD03754D03E599B4FC03754D04E544
:100CC20099B4FA03754D05E599B4FB06754E011208
:100CD200472EE599B4F906754E0412472EE599B4EC
:100CE200F73312472EC29C74AB900050F01206DA12
:100CF20074AA900050F09008F6E0B401051207853E
:100D020080031208C3900050E4F0D29C754E007527
:100D12004D007599F7E599D394E54007E599C39499
:100D2200F04002801685994F754E027E017F00E5E4
:100D32004FC394E61270CF8E328F33900895E4F051
:100D4200A3F0E599D394C24007E599C394E6400223
:100D5200802885994F754E0374E5C3954FF5337519
:100D62003200AE32AF33906A5612709EE493F8743A
:100D72000193900895C8F0A3C8F0D2990210DF90B1
:100D820008AAE0700AA220B35005A221B340028053
:100D92005C900895E0FEA3E0FF74FFBE00039F5045
:100DA20009EFC39446EE9406402B900895E0FEA30B
:100DB200E0FFEFD3946DEE94064009EFC394EEEE9C
:100DC20094064011900895E0FEA3E0FFEFD394FF54
:100DD200EE94064013900895E0FEA3E0FF90008792
:100DE200120048E599F08003859974801190089566
:100DF200E0FEA3E0FF900087120048E599F090081A
:100E0200951270DD900895E0FEA3E0FFEFB40106B5
:100E1200EEB407028003020EDA900787E0B43C02C8
:100E22008003020EDAA220B35005A221B340028051
:100E320055C29C1203BD900094E09008F5F0124058
:100E420012900173E09008ABF0900174E09008AC4E
:100E5200F0900175E09008ADF074AB900050F01284
:100E620006DA74AA900050F09008F6E0B401051278
:100E7200078580031208C39008F6E09000D0F09036
:100E82000050E4F08047C29C12019C74009008ABB1
:100E9200F074009008ACF074009008ADF0900094EB
:100EA200E09008F5F012401274AB900050F0120678
:100EB200DA74AA900050F01207851208C3D29C750A
:100EC20099FB75096475080012062480FED29C7590
:100ED2004E00754D007599FB0210DF900895E0FEFB
:100EE200A3E0FFEF4E7006859931753000900895AA
:100EF200E0FEA3E0FF74016F4E701BAC30AD31AA6F
:100F020032AB33ED2BFBEC3AFA8A068B0790008763
:100F1200120048E599F09008951270DD900895E06E
:100F2200FEA3E0FF74026F4E7021AC30AD317456F7
:100F32006D4C7006E54F64E66002800312472E1284
:100F42004012854F99754E00754D000210DF9008D2
:100F520095E0FEA3E0FF900087120048E599F0902B
:100F620008951270DD900895E0FEA3E0FFAC32AD6B
:100F7200338F028E038C068D07906A9C12709EE45A
:100F820093F9740193FEEAD39EEB994009854F9938
:100F9200754E00754D000210DF900895E0FEA3E04B
:100FA200FF900087120048E599F09008951270DDD5
:100FB200900895E0FEA3E0FFEFB40006EEB4010254
:100FC20080030210DF900066E0D394C7400B9000CC
:100FD20066E0C394C8F550801A900066E0D394632B
:100FE200400B900066E0C39464F550800690006662
:100FF200E0F550E55075F002A4FFAEF08F73EF906C
:101002000087127100EFFCE0FDEC90008A12710083
:10101200EDFCE0FDEC2DB5500280030210D10FEF84
:10102200900087127100E573FFE0FCEF90008B12D5
:101032007100ECFFE0FCEFC39CB55002800302108C
:10104200D1E573900089127100E573FFE0FCEF9027
:10105200008C127100ECFFE0FCEF2CB55071E573CF
:1010620090008D127100E0C395509008E3F0E57393
:1010720090008E127100E0C395509008E4F0E57381
:10108200900091127100E0C395509008E5F0E5736D
:10109200900092127100E0C395509008E6F0E5735B
:1010A200900093127100E0C395509008E7F0E57349
:1010B200900094127100E0C395509008E8F0120677
:1010C200507599F975096475080012062480FE7539
:0D10D20099FF75096475080012062480FE60
:0F3CC700020C9E020D81020EDD020F50020F9BB8
:1010DF0022E54D903CD6F82828730211C49008954C
:1010EF00E0FEA3E0FF900056120048E0F59990084B
:1010FF00951270DD900895E0FEA3E0FF741C6F4E13
:10110F007003754D000211C4856E990211C49008C9
:10111F0095E0FEA3E0FF900087120048E0F599EFFD
:10112F00B40107EEB40703754D009008951270DDFA
:07113F000211C4900896E0C4
:0F3CD6000210E90210EC02111702111D02114237
:10114600903D48F82828738552998067855F998075
:1011560062856199805D8565998058856799805318
:10116600856899804E8569998049856A99804490F9
:10117600001BE0F599803CA22BB340077599FAC293
:101186002B8017A21FB3400575990F800B90005452
:10119600E0F599900054E4F0C21F8017856B9980A2
:1011A60012856699800D856C9980087599FC800377
:0311B600754D0074
:103D480002114D02115202115702115C0211610257
:103D5800116602116B02117002117502117D0211B8
:0D3D6800A20211A70211AC0211B10211B6A6
:0B11B9009008951270DD8003123F16B5
:033CE5000211C108
:1011C40022E537255AFFAE5950010E9000871200D0
:1011D40048E0F538E537255AFFAE5950010E0FBFE8
:1011E40000010E900087120048E0F539853F3BE589
:1011F40038B539058538378041E539D39538401DF0
:10120400E539C39538853AF0A4FFAEF0E53B8E048A
:101214008F05FF1270BFED2538F537801DE538C303
:101224009539853AF0A4FFAEF0E53B8E048F05FFB7
:101234001270BFEDF4042538F53722E539D395381B
:10124400401DE539C39538853AF0A4FFAEF0E53B7F
:101254008E048F05FF1270BFED2538F537801DE52C
:1012640038C39539853AF0A4FFAEF0E53B8E048F80
:1012740005FF1270BFEDF4042538F5372290008D78
:10128400E0B4017FE56775F00A84FF7E008F37E5DF
:101294006775F00A84ADF07C008D3A753F0A755984
:1012A40005755A24E537C3941150051211C58006FB
:1012B4009005BCE0F537E537C394F05008E5379066
:1012C4000077F0800674EF900077F0E56775F00A18
:1012D40084FF7E008F37E56775F00A84ADF07C00EB
:1012E4008D3A753F0A755905755A5AE537C39411F5
:1012F40050051211C580069005F2E0F537E53790E8
:10130400004FF02290008DE0B40102800302139696
:10131400E56775F00A84FF7E008F37E56775F00A8C
:1013240084ADF07C008D3A753F0A755905755A36BF
:10133400E537C3941150051211C580069005CEE01F
:10134400F537E537C394F0500585374B8003754B6B
:10135400EFE56775F00A84FF7E008F37E56775F067
:101364000A84ADF07C008D3A753F0A755905755AAB
:1013740048E537C3941150051211C580069005E065
:10138400E0F537E537C394F0500585374C80037595
:101394004CEF22E55F75F00484FF7E008F37E55F34
:1013A40075F00484ADF07C008D3A753F04755901E5
:1013B400755A00E537C3943F50051211C580069055
:1013C40001C6E0F537E53790088FF8E4F0E8A3F0BC
:1013D400900053E075F020A4FFAEF09000D8E08EAA
:1013E400048F05FF1270BF8D379000C0E0D3955F66
:1013F40050030214A29000E4E0D3955F4010ED90F6
:1014040001C7127100E0F52B752A0002149F9000A9
:10141400AFE0D3955F4043E5379001C7127100E018
:10142400F538E5379001E7127100E0F5399000E4F2
:10143400E0F404255FF53A9000AFE0FE9000E4E0AC
:10144400F4042EF53BE538B53905853837800312A9
:10145400123F85372B752A008041E5379001E7124A
:101464007100E0F538E537900207127100E0F539B4
:101474009000AFE0F404255FF53A9000C0E0FE90E0
:1014840000AFE0F4042EF53BE538B539058538376F
:10149400800312123F85372B752A000215499000EC
:1014A400E7E0D3955F5011E537900247127100E0F1
:1014B400F52B752A000215499000B0E0D3955F50D2
:1014C40043E537900227127100E0F538E5379002C2
:1014D40047127100E0F5399000B0E0F404255FF59F
:1014E4003A9000E7E0FE9000B0E0F4042EF53BE50E
:1014F40038B53905853837800312123F85372B7587
:101504002A008041E537900207127100E0F538E5C2
:1015140037900227127100E0F5399000C0E0F4041E
:10152400255FF53A9000B0E0FE9000C0E0F4042E90
:10153400F53BE538B53905853837800312123F8508
:10154400372B752A00229000F8E0F53C753F1175A1
:101554005902755A00AE51AF52E53C75F00FA4FD27
:10156400ACF0EDD39FEC9E4021E53C8E048F05FF4B
:101574001270BFED75F010A4FFAEF0E55F75F011C9
:1015840084FD7C00ED2FF53D800EE55F75F0118440
:10159400FF7E00EF24F0F53D853D37E55F75F011E2
:1015A40084AFF07E008F3A1211C585373EAE51AF3D
:1015B400529000F8E075F00FA4FDACF0EDD39FEC71
:1015C4009E4028755902755A10853D371211C585FC
:1015D4003E38853739AE51AF52E53C8E048F05FF56
:1015E4001270EA8D3A853C3B12123FE53790088F22
:1015F400F8E4F0E8A3F0752B64752A00229000F853
:10160400E0F53C753F11755902755A00AE51AF5261
:10161400E53C75F00FA4FDACF0EDD39FEC9E4021AA
:10162400E53C8E048F05FF1270BFED75F010A4FF2A
:10163400AEF0E56175F01184FD7C00ED2FF53D8081
:101644000EE56175F01184FF7E00EF24F0F53D8511
:101654003D37E56175F01184AFF07E008F3A1211C9
:10166400C585373EAE51AF529000F8E075F00FA437
:10167400FDACF0EDD39FEC9E4028755902755A10CD
:10168400853D371211C5853E38853739AE51AF5285
:10169400E53C8E048F05FF1270EA8D3A853C3B12BF
:1016A400123FE53790088FF8E4F0E8A3F0E56B60AB
:1016B40017E56BC394FE50109000ECE0B40209905F
:1016C40000DAE0D3940B5002801F90088FE0FEA351
:1016D400E0FFE56B1270CF74E78E048F05FF127084
:1016E400BF90088FECF0A3EDF09000C2E0B4045F6B
:1016F400E55F75F00484FF7E008F37E55F75F004C5
:1017040084ADF07C008D3A753F04755901755A001B
:10171400E537C3943F50051211C580069001C6E019
:10172400F53790088FE0FEA3E0FFE5371270CF7421
:10173400328E048F05FF1270BF90088FE0FEA3E085
:10174400FFEF2DFDEE3CFC90088FECF0A3EDF0755F
:101754002B64752A002290008DE0B40146E567757C
:10176400F00A84FF7E008F37E56775F00A84ADF0D8
:101774007C008D3A753F0A755905755A00E537C3E3
:10178400941150051211C58006900598E0F537AE06
:101794002AAF2BE5372FFF50010E74641271128E9D
:1017A4002A8F2B90008EE0B40146E56875F00A8418
:1017B400FF7E008F37E56875F00A84ADF07C008DFC
:1017C4003A753F0A755905755A6CE537C39411503B
:1017D400051211C58006900604E0F537AE2AAF2B3A
:1017E400E5372FFF50010E74641271128E2A8F2B6D
:1017F40090009DE0B40249E56AC3944175F0058404
:10180400FF7E008F37E56A75F00584ADF07C008DAE
:101814003A753F05755906755A00E537C394135058
:10182400051211C5800690069AE0F537AE2AAF2B53
:10183400E5372FFF50010E74641271128E2A8F2B1C
:101844009000DFE0B4020280030218F9E55F75F04E
:101854001584FF7E008F37E55F75F01584ADF07C4D
:10186400008D3A753F15755903755AF4E537C394DD
:101874000B50051211C58006900486E0F537E53754
:1018840075F0FFA4FFAEF09000E0E08E048F05FF3A
:101894001270BFED900074F0E56675F078A4FFAEA9
:1018A400F074FF8E048F05FF1270BF8C598D5A742B
:1018B400028C068D071200398F37AC59AD5A740467
:1018C400FF1270EA8D3A753F04755906755A28E57A
:1018D40037C3941D50051211C580069006CCE0F55F
:1018E40037AE2AAF2BE5372FFF50010E7464127107
:1018F400128E2A8F2B90008CE0B4025DE56175F0A6
:1019040064A4FFAEF074081200398E5B8F5C74051A
:101914008E048F05FF1270BF8D37AE5BAF5C74050C
:101924008E048F05FF1270EA8D3A753F05755905CF
:10193400755ADEE537C3941350051211C58006901D
:101944000678E0F537AE2AAF2BE5372FFF50010EAE
:1019540074641271128E2A8F2B9000CEE0707F90E7
:101964000053E075F00A84FF7E008F37900053E047
:1019740075F00A84ADF07C008D3A753F0A755905FF
:10198400755AC0E537C3940E50051211C5800690F0
:101994000655E0F537E537900078F09000EDE0B4B7
:1019A400023C900053E075F00A84FF7E008F37906C
:1019B4000053E075F00A84ADF07C008D3A753F0A5F
:1019C400755905755ACFE537C3940E50051211C5E4
:1019D4008006900664E0F537E537900079F02290B0
:1019E4000095E0B401179008EAE0252BFFAE2A50D9
:1019F400010E9000E9E01271128E2A8F2B90010DD6
:101A0400E0B4011490010EE0A851B80004955250BE
:101A140007E55FC39560400280139000B7E0252B73
:101A2400FFAE2A50010E8E2A8F2B021E4A9000957B
:101A3400E0B40306A228B3B3400280509008F4E057
:101A440070109008EDE0C39405A851B800069552B3
:101A5400400280109000B7E0252BFFAE2A50010E03
:101A64008E2A8F2B9008F4E0600D9008EDE0A851C9
:101A7400B800069552400280109000B7E0252BFF75
:101A8400AE2A50010E8E2A8F2B021E4A90008FE040
:101A9400B402028003021E4A900092E0602FE567C0
:101AA400D394464028900012E0FEA3E0FF9000CDBE
:101AB400E075F003A4FDACF0EFD39DEE9C400E90D6
:101AC40000F1E0A851B80005D395525003021E4A14
:101AD4009000C2E0B403028003021C9285615A752F
:101AE4005900900099E0A851B800049552500E9006
:101AF400009AE0A859B80005D3955A5003021C8FE8
:101B0400E56175F002A4FFAEF074158E048F05FF35
:101B14001270BF8C068D07900617120048FEE0FF76
:101B2400EE900091E0FEEF8E0088F0A4FFAEF0741A
:101B3400648E048F05FF1270BF8C598D5A90005328
:101B4400E075F018A4FFAEF09000D8E08E048F0585
:101B5400FF1270BF8C068D0790062F120048AE59F5
:101B6400AF5AE01270CF74648E048F05FF1270BFF9
:101B74008C598D5AE565A859B80005D3955A500378
:101B8400021C06E565C3955AFFE49559FE8E598FEC
:101B94005A7428BE00039F500C755A287559007456
:101BA4000D900054F0AE59AF5A900092E01270CFED
:101BB40074288E048F05FF1270BF8C598D5A9008BB
:101BC4008FE0FEA3E0FF740A8E048F05FF1270BF3E
:101BD4008D068C07AC59AD5ACFCECF120003740AD0
:101BE4008E048F05FF1270BF8C598D5A90088FE0B8
:101BF400FEA3E0FF12711A90088FEEF0A3EFF0023B
:101C04001C8FE565A859B80004955A507EAE59AFAB
:101C14005AE5651271128E598F5A7428BE00039FBB
:101C2400500C755A28755900740D900054F0AE5933
:101C3400AF5A900092E01270CF74288E048F05FF83
:101C44001270BF8C598D5A90088FE0FEA3E0FF7488
:101C54000A8E048F05FF1270BF8D068C07AC59AD38
:101C64005ACFCECF120003740A8E048F05FF127070
:101C7400BF8C598D5A90088FE0FEA3E0FFEF2DFD35
:101C8400EE3CFC90088FECF0A3EDF0021E4A9000AD
:101C9400DAE0855FF0A4FFAEF074051270CF74072C
:101CA4001200398E598F5A900099E0A851B8000457
:101CB4009552501290009AE075F002A4FDACF0EF3A
:101CC400C39DEE9C4003021E4AE55F75F00B84FF42
:101CD4007E00900617120048FEE0FFEE900091E0AF
:101CE400FEEF8E0088F0A4FFAEF074648E048F05BE
:101CF400FF1270BF8C598D5A900053E075F018A4F0
:101D0400FFAEF09000D8E08E048F05FF1270BF8CF8
:101D1400068D0790062F120048AE59AF5AE0127094
:101D2400CF74648E048F05FF1270BF8C598D5AE5F1
:101D340065A859B80005D3955A5003021DC1E5653D
:101D4400C3955AFFE49559FE8E598F5A7428BE00E4
:101D5400039F500C755A28755900740D900054F067
:101D6400AE59AF5A900092E01270CF74288E048F4F
:101D740005FF1270BF8C598D5A90088FE0FEA3E0C6
:101D8400FF740A8E048F05FF1270BF8D068C07AC9A
:101D940059AD5ACFCECF120003740A8E048F05FFBB
:101DA4001270BF8C598D5A90088FE0FEA3E0FF1289
:101DB400711A90088FEEF0A3EFF0021E4AE565A8B1
:101DC40059B80004955A507EAE59AF5AE565127160
:101DD400128E598F5A7428BE00039F500C755A28CE
:101DE400755900740D900054F0AE59AF5A9000929A
:101DF400E01270CF74288E048F05FF1270BF8C59C7
:101E04008D5A90088FE0FEA3E0FF740A8E048F05BC
:101E1400FF1270BF8D068C07AC59AD5ACFCECF12CE
:101E24000003740A8E048F05FF1270BF8C598D5AFB
:101E340090088FE0FEA3E0FFEF2DFDEE3CFC900840
:101E44008FECF0A3EDF0229000EDE0B4027BE55FAF
:101E540075F00884FF7E008F37E55F75F00884AD68
:101E6400F07C008D3A753F08755901755AE0E537E5
:101E7400C3943F50051211C58006900286E0F537E1
:101E8400E537900891F8E4F0E8A3F0900891E0FEBB
:101E9400A3E0FFAC2AAD2B12000374648E048F05FB
:101EA400FF1270BF900891ECF0A3EDF090008AE06F
:101EB4008C068D071270CF74648E048F05FF127028
:101EC400BF900891ECF0A3EDF090088FE0FEA3E042
:101ED400FFAC2AAD2B12000374648E048F05FF122D
:101EE40070BF90088FECF0A3EDF090008AE08C06B0
:101EF4008D071270CF74648E048F05FF1270BF902B
:101F0400088FECF0A3EDF0A204401DAE51AF527463
:101F140005BE00039F5002D204E561D394CC40086F
:101F2400D2027411900054F0229000ECE0B4020844
:101F34009000DAE0640B6002804590088FE0FEA315
:101F4400E0FFE56B1270CF74E78E048F05FF12700B
:101F5400BF90088FECF0A3EDF09000EDE0B4021F09
:101F6400900891E0FEA3E0FFE56B1270CF74E78E5A
:101F7400048F05FF1270BF900891ECF0A3EDF09070
:101F840000ACE05402601B9000A3E0A851B800121A
:101F9400D39552400DA204B3B35007E561C3949A9C
:101FA4004002805FAE34AF359000A1E075F002A42A
:101FB400FDACF0EF2DFDEE3CFC74022DFD50010C48
:101FC400E561BC003ED39D403A754301A22F4033E6
:101FD4009000A2E075F05EA4FDACF07405FF1270F1
:101FE400BF8C5B8D5C124AA390088FE0FEA3E0FFD8
:101FF4009000A2E02FFF50010E90088FEEF0A3EFA7
:10200400F0D22FE561A834B8000495355002C22FF0
:10201400856135753400E54370030221239000FF88
:10202400E0C39543500302211590010FE0C39402CD
:1020340040030220BFE56775F00A84FF7E00900527
:1020440087120048E0F55A755900AE59AF5A90000E
:10205400A2E01270CF74648E048F05FF1270BF8CDF
:102064005B8D5C9000FFE004C395438C068D0712E2
:1020740070CF9000FFE08E048F05FF1270BF8C5B61
:102084008D5C90088FE0FEA3E0FFEF2DFDEE3CFC9D
:1020940090088FECF0A3EDF09000EDE0B4021A90FC
:1020A4000891E0FEA3E0FFAA5BAB5CEF2BFBEE3AEA
:1020B400FA900891EAF0A3EBF080569000FFE00458
:1020C400C39543854BF0A4FFAEF09000FFE08E046F
:1020D4008F05FF1270BF8C5B8D5C90088FE0FEA3B0
:1020E400E0FFEF2DFDEE3CFC90088FECF0A3EDF04B
:1020F4009000EDE0B4021A900891E0FEA3E0FFAA7C
:102104005BAB5CEF2BFBEE3AFA900891EAF0A3EBA1
:10211400F005439000FFE0C39543500375430090DE
:1021240000ACE05401601B9000A0E0A851B800127C
:10213400D39552400DA204B3B35007E55FC394CCCA
:102144004002806090009EE075F003A4FFAEF0E5CD
:10215400402FFF50010E74032FFF50010EE55FBEA8
:102164000042D39F403E754401A22F403790009F08
:10217400E075F05EA4FFAEF074058E048F05FF12C7
:1021840070BF8C5B8D5C124AA390088FE0FEA3E0C5
:10219400FF90009FE02FFF50010E90088FEEF0A3F8
:1021A400EFF0D22FE55FC395405002C22F855F4008
:1021B400E54470030222BD900100E0C3954450033E
:1021C4000222AF90010FE0C394024003022259E5BA
:1021D4006775F00A84FF7E00900587120048E0F5D9
:1021E4005A755900AE59AF5A90009FE01270CF74DF
:1021F400648E048F05FF1270BF8C5B8D5C900100B0
:10220400E004C395448C068D071270CF900100E062
:102214008E048F05FF1270BF8C5B8D5C90088FE07D
:10222400FEA3E0FFEF2DFDEE3CFC90088FECF0A345
:10223400EDF09000EDE0B4021A900891E0FEA3E006
:10224400FFAA5BAB5CEF2BFBEE3AFA900891EAF045
:10225400A3EBF08056900100E004C39544854CF054
:10226400A4FFAEF0900100E08E048F05FF1270BF52
:102274008C5B8D5C90088FE0FEA3E0FFEF2DFDEEFC
:102284003CFC90088FECF0A3EDF09000EDE0B4027C
:102294001A900891E0FEA3E0FFAA5BAB5CEF2BFB76
:1022A400EE3AFA900891EAF0A3EBF00544900100AD
:1022B400E0C39544500375440090088FE0FEA3E00A
:1022C400FF9000B1E0BE00039F500D9000B1E0907C
:1022D400088FF8E4F0E8A3F09000EDE0B402129067
:1022E4000891E0FEA3E0FF9000B1E0BE00059F402E
:1022F40002800D9000B1E0900891F8E4F0E8A3F0BA
:10230400229000EDE0B401028003022453A204B33E
:10231400500302243A9000B8E0B4017A90088FE0A8
:10232400FEA3E0FFAC51AD52120003743C8E048F47
:1023340005FF1270BF9000C8E0BC00159D401290CC
:10234400088FE0FEA3E0FF9000CAE0BE00039F50A8
:1023540002D20390088FE0FEA3E0FFAC51AD52120D
:102364000003743C8E048F05FF1270BF9000C8E018
:10237400C3940ABC001AD39D401690088FE0FEA3B4
:10238400E0FF9000CAE0C39405BE0004D39F50024E
:102394008002C203807A90088FE0FEA3E0FFAC5174
:1023A400AD5212000374788E048F05FF1270BF9033
:1023B40000C8E0BC00159D401290088FE0FEA3E029
:1023C400FF9000CAE0BE00039F5004D203804190F6
:1023D400088FE0FEA3E0FFAC51AD52120003747805
:1023E4008E048F05FF1270BF9000C8E0C3940ABC2E
:1023F400001AD39D401690088FE0FEA3E0FF9000E2
:10240400CAE0C39405BE0004D39F50028002C203F5
:10241400A203B3402190088FE0FEA3E0FF9000C91F
:10242400E01270CF74648E048F05FF1270BF9008A1
:102434008FECF0A3EDF0A203B3400CA2334006747A
:1024440024900054F0D233A2034002C2338002C26B
:102454000390004FE06006A204B3B34002801990D9
:10246400088FE0FEA3E0FF90004FE02FFF50010E25
:1024740090088FEEF0A3EFF0A201B34006A202B3DE
:10248400B3500990001AE4F0A3F0802D90088FE077
:10249400FEA3E0FF7400D39F74019E401190088F47
:1024A400E0F8A3E090001AC8F0A3C8F0800B74FF12
:1024B40090001AF8E4F0E8A3F09000CFE0C394048D
:1024C400400C9008F1E0C3940240030225AD900053
:1024D400B8E0B4014790088FE0FEA3E0FF745E12F9
:1024E40070CF74058E048F05FF1270BF90088FECB7
:1024F400F0A3EDF09000EDE0B4021F900891E0FE2F
:10250400A3E0FF745E1270CF74058E048F05FF1272
:1025140070BF900891ECF0A3EDF0804590088FE037
:10252400FEA3E0FF745E1270CF740A8E048F05FF61
:102534001270BF90088FECF0A3EDF09000EDE0B4C2
:10254400021F900891E0FEA3E0FF745E1270CF7446
:102554000A8E048F05FF1270BF900891ECF0A3ED72
:10256400F090088FE0FEA3E0FF7402BE000CD39F3E
:102574004008752902752800800A90088FE0F52824
:10258400A3E0F529900891E0FEA3E0FF7402BE00E9
:102594000CD39F4008752D02752C00800A90089179
:1025A400E0F52CA3E0F52D804690088FE0FEA3E033
:1025B400FF7401BE000CD39F4008752901752800E3
:1025C400800A90088FE0F528A3E0F529900891E0AF
:1025D400FEA3E0FF7401BE000CD39F4008752D01DB
:1025E400752C00800A900891E0F52CA3E0F52D905D
:1025F4000018E528F0A3E529F0A236B34009C2018A
:1026040090001AE4F0A3F022900053E090038712A4
:102614007100E0F541754264900053E0FE9000C300
:10262400E0D39E4037E55F75F00884FF7E008F3766
:10263400E55F75F00884ADF07C008D3A753F087550
:102644005903755A96E537C3941F50051211C58076
:102654000690043CE0F5378537428035E55F75F038
:102664000884FF7E008F37E55F75F00884ADF07C49
:10267400008D3A753F08755903755AB6E537C3940A
:102684001F50051211C5800690045CE0F5378537AC
:1026940042229000F9E0F53C753F11755904755AD2
:1026A40000AE51AF52E53C75F00FA4FDACF0EDD394
:1026B4009FEC9E4021E53C8E048F05FF1270BFED18
:1026C40075F010A4FFAEF0E55F75F01184FD7C0099
:1026D400ED2FF53D800EE55F75F01184FF7E00EF70
:1026E40024F0F53D853D37E55F75F01184AFF07E4C
:1026F400008F3A1211C585373EAE51AF529000F9A2
:10270400E075F00FA4FDACF0EDD39FEC9E4028756E
:102714005904755A10853D371211C5853E388537E1
:1027240039AE51AF52E53C8E048F05FF1270EA8D2D
:102734003A853C3B12123F85374175426422900032
:10274400F9E0F53C753F11755904755A00AE51AF67
:1027540052E53C75F00FA4FDACF0EDD39FEC9E4028
:1027640021E53C8E048F05FF1270BFED75F010A4B7
:10277400FFAEF0E56175F01184FD7C00ED2FF53DB1
:10278400800EE56175F01184FF7E00EF24F0F53DC5
:10279400853D37E56175F01184AFF07E008F3A1204
:1027A40011C585373EAE51AF529000F9E075F00F78
:1027B400A4FDACF0EDD39FEC9E4028755904755AE6
:1027C40010853D371211C5853E38853739AE51AF76
:1027D40052E53C8E048F05FF1270EA8D3A853C3B2E
:1027E40012123F8537417542649000F4E0B40479D5
:1027F400900053E0FE9000C3E0D39E4037E55F7540
:10280400F00884FF7E008F37E55F75F00884ADF033
:102814007C008D3A753F08755903755A96E537C3A0
:10282400941F50051211C5800690043CE0F53785CD
:1028340037428035E55F75F00884FF7E008F37E509
:102844005F75F00884ADF07C008D3A753F087559CA
:1028540003755AB6E537C3941F50051211C5800697
:1028640090045CE0F5378537422290008DE0B40196
:102874003BE56775F00A84FF7E008F37E56775F0E6
:102884000A84ADF07C008D3A753F0A755905755A76
:1028940012E537C3941150051211C580069005AA9C
:1028A400E0F537E5422537C39464F54290008EE0A5
:1028B400B4013BE56875F00A84FF7E008F37E56854
:1028C40075F00A84ADF07C008D3A753F0A755905A0
:1028D400755A7EE537C3941150051211C5800690D0
:1028E4000616E0F537E5422537C39464F542E54121
:1028F4002542F536900095E0B402109008E9E025F1
:1029040036FE9000E9E0F4042EF5369000ECE0D3B6
:1029140094014040E56BC394E7501D74E7C3956B85
:10292400FE9008EBE08E00F5F0E884FF7E008F3720
:10293400E5362537F536801CE56BC394E7FE900831
:10294400EBE08E00F5F0E884FF7E008F37E536C3B8
:102954009537F536A2044006E5412464F536E5369C
:10296400D394644009E536C39464F5368003753620
:10297400009000C5E0C3953650069000C5E0F536DA
:1029840022D201900076E0A851B800049552503E3E
:10299400900076E0A851B800049552500375360FA4
:1029A400900076E004A851B800049552500375369F
:1029B40007900076E02402A851B800049552500212
:1029C400C201900076E060067409900054F0C22EB3
:1029D4007E017F009000CBE01270CF9000DAE08E91
:1029E400048F05FF1270BFE55FBC000CD39D400847
:1029F400D236740A900054F090008DE0B40109902E
:102A040000CCE0C39567400280159000DEE0A85139
:102A1400B8000495525002C201740B900054F09017
:102A2400008DE0B40107E567C394644002801D9003
:102A34000124E0600D900124E0A851B800069552ED
:102A440040028008C201740B900054F0A2014003BC
:102A5400753600C23590010DE0B4011490010EE00A
:102A6400A851B8000495525007E55FC39560400231
:102A7400802A9000B6E0D3941D400B9000B6E0C3CA
:102A8400941EF5368003753600A232400874159002
:102A94000054F0D235D232D230022B7FC230C2324F
:102AA400900095E0B40306A228B3B34003022B7F41
:102AB4009008EDE0C39405A851B80004955250065F
:102AC4009008F4E06002801F9000B6E0D3941D40AB
:102AD4000B9000B6E0C3941EF5368003753600747F
:102AE4000C900054F0D2359008EDE0A851B80004E1
:102AF400955250069008F4E07002801F9000B6E0F2
:102B0400D3941D400B9000B6E0C3941EF5368003A9
:102B1400753600740C900054F0D2359008EDE0A89E
:102B240051B80004955250319000D4E0B40228D238
:102B34002E9008F3E0FE9008F4E0D39E500690082F
:102B4400F4E0700280099008F3E4F0C22E8006904D
:102B540008F3E004F08002C2019008EDE02405A827
:102B640051B80004955250139000D4E0B4020A9076
:102B740008F4E07002D22E8002C201A22DB34027D5
:102B84009000B6E0D3941D400B9000B6E0C3941EB1
:102B9400F5368003753600A2314006741090005457
:102BA400F0D231D2358002C23185366C9000B6E065
:102BB400D3941D4018900084E02536FE900053E025
:102BC40075F01E84FC7F00EE2CF5368037A235B3F9
:102BD4004016900084E0FE900053E075F01E84FCE3
:102BE4007F00EE2CF536801C900086E02536FE90A2
:102BF4000084E02EFE900053E075F01E84FC7F00FC
:102C0400EE2CF536A236B34005D22E756C00229018
:102C14000053E075F00584FF7E008F37900053E089
:102C240075F00584ADF07C008D3A753F0575590348
:102C3400755AD69000D8E01475F00584FF7E00E53F
:102C440037BE00039F50051211C5800BE537900471
:102C54005D127100E0F537E5379008ECF09008EC70
:102C6400E0FE9000C7E0C39E50089000C7E09008C3
:102C7400ECF09000B6E0D3941D401E9008ECE0FE0A
:102C8400900084E02EFE900053E075F01E84FC7FDB
:102C940000EE2C9008ECF0803FA235B34018900071
:102CA40084E0FE900053E075F01E84FC7F00EE2C5F
:102CB4009008ECF080229008ECE0FE900086E02E74
:102CC400FE900084E02EFE900053E075F01E84FC1C
:102CD4007F00EE2C9008ECF02290008DE0B40136D9
:102CE400E56775F00A84FF7E00900587120048E0CE
:102CF400F546E546D394644010E546C3946475F004
:102D04000F84FF7E008F4680037546009000AAE082
:102D14002546F54680069000AAE0F54622E567754B
:102D2400F00A84FF7E00900587120048E0C394698E
:102D34004007E567D3946440559000F4E0C39403DE
:102D44005026900889E0FEA3E0FF7404120039E5E0
:102D54005F1270CF740F8E048F05FF1270BF90083E
:102D640087ECF0A3EDF08024900889E0FEA3E0FF57
:102D74007404120039E5611270CF740F8E048F054C
:102D8400FF1270BF900887ECF0A3EDF0800F90085D
:102D940089E0F8A3E0900887C8F0A3C8F0A2044033
:102DA4001A900889E0FEA3E0FF74031270CF740147
:102DB400120039900887EEF0A3EFF090009DE0B484
:102DC4000262E56AC3944175F00584FF7E008F3783
:102DD400E56A75F00584ADF07C008D3A753F0575A4
:102DE4005906755A14E537C3941750051211C58056
:102DF400069006AEE0F537900887E0FEA3E0FF7486
:102E04000A8E048F05FF1270BFE5378C068D0712FA
:102E140070CF740A8E048F05FF1270BF900887EC80
:102E2400F0A3EDF0900887E0FEA3E0FF90088DE0AA
:102E3400FCA3E0FDEDD39FEC9E400F90088DE0F8DD
:102E4400A3E0900887C8F0A3C8F022E50875F00451
:102E5400A4FFAEF09006CA120048E0903CE8F828BF
:102E64002873804C85527380479000DAE0855FF0C8
:102E7400A4FFAEF074081200398F73803385617338
:102E8400802E8567738029856873802485697380A3
:102E94001F856A73801A856B73801585667380102D
:102EA400856573800B856C73800690001BE0F57359
:103CE800022E66022E68022E6D022E81022E860298
:103CF8002E8B022E90022E95022E9A022E9F022EB5
:073D0800A4022EA9022EAE59
:102EB400E50875F004A4FFAEF09006CB120048E5D7
:102EC4000875F004A4FFAEF0E0FC9006CC120048B4
:102ED400ECFEE0FFEEC39F4003022FBCE50875F053
:102EE40004A4FFAEF09006CA120048E0B40441E521
:102EF4000875F004A4FFAEF09006CC120048E0C3BD
:102F04009573500AE508F50CD39237123E43E50851
:102F140075F004A4FFAEF09006CB120048E0D39500
:102F240073400AE508F50CC39237123E43022FBAE8
:102F3400E50875F004A4FFAEF09006CB120048E05B
:102F4400C395735015E50875F004A4FFAEF0900620
:102F5400CC120048E0D395735002800AE508F50CC2
:102F6400D39237123E43E50875F004A4FFAEF09007
:102F740006CB120048E0D395735015E50875F004AC
:102F8400A4FFAEF09006CC120048E0C39573500A3B
:102F9400E508F50CC39237123E439006D2E0B40123
:102FA400099000E6E0D395615002800A7402F50CA2
:102FB400C39237123E43806AE50875F004A4FFAE5D
:102FC400F09006CB120048E0D395734015E50875E0
:102FD400F004A4FFAEF09006CC120048E0C3957351
:102FE4004002800AE508F50CC39237123E43E50817
:102FF40075F004A4FFAEF09006CB120048E0C39530
:10300400734015E50875F004A4FFAEF09006CC12E9
:103014000048E0D39573400AE508F50CD3923712C3
:103024003E4322AE2EAF2F74C9BE000CD39F40087E
:10303400782E127122023141752F01752E00AE5186
:10304400AF52E546BE000DD39F40099000BCE0D3CB
:10305400954740028023754700E546C39552F573B2
:103064009000BFE0D395454008E5452573F54580BC
:10307400069000BFE0F54580020547900098E0D334
:103084009561401CE55FC395604015AE51AF52E5B4
:1030940046BE00039F50099000BDE0D3954840020E
:1030A400806E9008EEE0A851B80004955250037564
:1030B4004A009008EEE0A851B8000BD395524006A0
:1030C400E5529008EEF0E54A7041E552C39546F5A5
:1030D40073E573D3940540037573059000BEE0C394
:1030E40095455007E573C3954540028009E545C3FE
:1030F4009573F54580069000BEE0F5459000BEE06E
:10310400D3954540069000BEE0F545754800800221
:103114000548E54A7016900098E0C39561500DE5A6
:10312400462405A851B8000695524002800F90002D
:10313400ABE0F545754A0174789008EEF022AE2EA6
:10314400AF2F74E9D39F74039E4008782E12712226
:103154000232FB752F01752E00754532A229403DC0
:10316400E54775F00284AFF07E00EF4E70057545BB
:103174001980037545329000ABE075F002A4FFAEF0
:10318400F0E547BE0006D39F4002D2290547754AA1
:103194000374789008EEF07549000232E2AE51AF44
:1031A40052E5466F4E70030232E2E546BE000DD38F
:1031B4009F40099000BCE0D395474002800F7547BB
:1031C40000E54AC394035003754519800DE546C3D1
:1031D4009552F573E5472573F547900098E0D3952C
:1031E40061400E9008EEE0A851B80007D395524014
:1031F40002800C05499000ABE0B54903754A00E52F
:103204004AB40306A204B3B34002800A0549E5495F
:10321400B43C03754A02E54AB402299008EEE0A8DA
:1032240051B8000ED395524009E5529008EEF0755E
:103234004900900098E0C39561500975490074787D
:103244009008EEF0E54A705A900098E0D3956140FA
:103254001CE55FC395604015AE51AF52E546BE0014
:10326400039F50099000BDE0D39548400280087543
:10327400480075454B8028E552C39546F573E573C0
:10328400D394054003757305900098E0D39561408D
:1032940008E5482573F5488006E5482406F5487591
:1032A4004900E54A7016900098E0C39561500DE519
:1032B400462405A851B80006955240028003754A79
:1032C40001E54AB4011875451905499000ABE0B50C
:1032D4004906754A0275490074789008EEF0A20216
:1032E400B34003754532E54575F00AA4FFAEF0908E
:1032F4000893EEF0A3EFF022E56F903D0FF8282835
:1033040073023CA8900090E0700302362C9000C633
:10331400E0B4010280030234BF900051E0655E60B6
:1033240009E552455160030234BC7E017F00E5BECD
:103334001270CFE5BD2FFF50010E8E598F5A9001A8
:103344002BE075F010A4FDACF08C5B8D5CEFD39D8D
:10335400EE9C400912711A8E598F5A8006755A00D4
:10336400755900AE59AF5A740E1270CF9000BBE07D
:103374008E048F05FF1270BF900897ECF0A3EDF058
:10338400E56B600FE56BC394FE50089000ECE064BD
:1033940002600280649000DAE0B40B1F900897E0AA
:1033A400FEA3E0FF74E71270CFE56B8E048F05FF78
:1033B4001270BF900897ECF0A3EDF09000DAE0D320
:1033C400940B40089000C2E064046002802B9008D3
:1033D40097E0FEA3E0FF90089BE0FCA3E0FDEFD3A1
:1033E4009DEE9C400D12711A900897EEF0A3EFF039
:1033F4008007900897E4F0A3F0900897E0FEA3E01C
:10340400FFEFD39400EE94014008D2367426900066
:1034140054F0A236B3B3502C7E057F009000DAE05E
:103424008E048F05FF1270BF900897E0FEA3E0FFA3
:10343400EFC39DEE9C400FAC51AD52740FBC000421
:10344400D39D50028002C236900090E0B4022790CF
:103454000899E0FEA3E0FF900897E0FCA3E0FDEFED
:103464002DFDEE3CFC74018C068D0712003990088A
:1034740097EEF0A3EFF0900897E0FEA3E0FF90082A
:1034840099E0FCA3E0FDEDD39FEC9E4004D22C8098
:1034940002B22C900897E0F8A3E0900899C8F0A332
:1034A400C8F09000C2E064016006A22CB3B34002ED
:1034B4008006900898E0F55F02362AD22C7E017FC0
:1034C40000E5BE1270CFE5BD2FFF50010E8E598F5F
:1034D4005A90012BE075F010A4FDACF08C5B8D5C70
:1034E400EFD39DEE9C400912711A8E598F5A8006B3
:1034F400755A00755900AE59AF5A740E1270CF90B8
:1035040000BBE08E048F05FF1270BF900897ECF0AB
:10351400A3EDF0E56B600FE56BC394FE50089000DB
:10352400ECE06402600280649000DAE0B40B1F9067
:103534000897E0FEA3E0FF74E71270CFE56B8E04FA
:103544008F05FF1270BF900897ECF0A3EDF0900088
:10355400DAE0D3940B40089000C2E0640460028077
:103564002B900897E0FEA3E0FF90089BE0FCA3E00B
:10357400FDEFD39DEE9C400D12711A900897EEF06A
:10358400A3EFF08007900897E4F0A3F0900897E089
:10359400FEA3E0FFEFD39400EE94014008D236740A
:1035A40026900054F0A236B3B3502C7E057F0090D1
:1035B40000DAE08E048F05FF1270BF900897E0FEDA
:1035C400A3E0FFEFC39DEE9C400FAC51AD52740FCE
:1035D400BC0004D39D50028002C236900090E0B437
:1035E4000227900899E0FEA3E0FF900897E0FCA36F
:1035F400E0FDEF2DFDEE3CFC74018C068D071200FE
:1036040039900897EEF0A3EFF0900897E0F8A3E064
:10361400900899C8F0A3C8F09000C2E06401600665
:10362400900898E0F55F8003755F0090008CE0706F
:1036340006756F030232FC75BB18023CA8023CA855
:1036440090008CE070030237B57E017F00E5BE1266
:1036540070CFE5BD2FFF50010E8E598F5A9000D2C6
:10366400E0B4010F7E0F7FFFAC59AD5A12711A8E70
:10367400598F5A9000F7E0B40245AE59AF5A900002
:1036840024E0FCA3E0FDEDD39FEC9E400A900024CF
:10369400E559F0A3E55AF0AE59AF5A900026E0FC84
:1036A400A3E0FDEFD39DEE9C400A900026E559F07F
:1036B400A3E55AF0AE59AF5A74041200398F6190E1
:1036C40000F7E0704CAE59AF5A900024E0FCA3E040
:1036D400FDEFD39DEE9C400912711A8E598F5A80CA
:1036E40006755A00755900AE59AF5A74101270CF4E
:1036F4009000F6E08E048F05FF1270BF8C598D5A2E
:1037040074FFBC0009D39D4005855A61800375612F
:10371400FE9000C2E0B4010280030237B3A204B3F6
:10372400B3500E900096E0A851B80005D3955250BE
:103734000280719000D3E08561F0A4FFAEF0746460
:103744008E048F05FF1270BF8C598D5AE56B60167D
:10375400E56BC394FE500F9000ECE0B402089000B7
:10376400DAE0640B60028017AE59AF5A74E7127046
:10377400CFE56B8E048F05FF1270BF8C598D5AAE46
:1037840059AF5A900897E0FCA3E0FDEDD39FEC9E5F
:103794004005855A5F800BA22CB34006900898E040
:1037A400F55F800BA22CB34006900898E0F55F808B
:1037B4000375610090008FE07006756F050232FC9E
:1037C40075BB19023CA8023CA890008FE07003026C
:1037D400389CE55ED3955D400302389A900022E060
:1037E400FEA3E0FFE565127112900022EEF0A3EF54
:1037F400F09000FCE0B402247E017F00E5BE12706C
:10380400CFE5BD2FFF50010E8F048E057E0F7FFF85
:10381400CDCCCD12711A8E598F5A80147E017F003F
:10382400E5BE1270CFE5BD2FFF50010E8E598F5AA1
:103834009000FCE07017AE59AF5A740A1270CF743E
:10384400518E048F05FF1270BF8D658019AE59AF7C
:103854005A740A1270CF8F048E057E017F95CDCCE9
:10386400CD126FBD8F65E565D394644003756564BF
:10387400900022E0FEA3E0FFE5652FFF50010E90CB
:103884000022EEF0A3EFF0900093E0048E048F0585
:10389400FF1270BF8D6580037565329000DFE070A4
:1038A40006756F070232FC75BB13023CA8023CA8E4
:1038B4009000DFE0604A7E017F00E5BE1270CFE534
:1038C400BD2FFF50010E8E598F5A74041200398F88
:1038D400669000E1E08566F0A4FDACF07464FF122C
:1038E40070BF8D669000E0E08566F0A4FFAEF074D2
:1038F400FF8E048F05FF1270BFED900075F08003FA
:1039040075660090008DE07006756F090232FC75D3
:10391400BB17023CA8023CA890008DE0B4010280D1
:10392400030239B07E017F00E5BE1270CFE5BD2FE2
:10393400FF50010E8E598F5A9008EFE060199008DD
:10394400EFE014906AE212008CE493FC740193FD9E
:10395400EDC39FEC9E400280069008EFE014F090C7
:1039640008EFE0C394B3501DAE59AF5A9008EFE08E
:1039740004906AE212008CE493FC740193FDEFC39B
:103984009DEE9C400280069008EFE004F09008EF62
:10399400E0FE9000B3E08E0088F0A4FFAEF0746403
:1039A4008E048F05FF1270BF8D67800375670090CA
:1039B400008EE07006756F0B0232FC75BB16023C7C
:1039C400A8023CA890008EE0B401028003023A5C95
:1039D4007E017F00E5BE1270CFE5BD2FFF50010EC2
:1039E4008E598F5A9008F0E060199008F0E0149016
:1039F4006C4C12008CE493FC740193FDEDC39FECBA
:103A04009E400280069008F0E014F09008F0E0C3B5
:103A140094B3501DAE59AF5A9008F0E004906C4C2A
:103A240012008CE493FC740193FDEFC39DEE9C4063
:103A34000280069008F0E004F09008F0E0FE9000A8
:103A4400B9E08E0088F0A4FFAEF074648E048F0594
:103A5400FF1270BF8D68800375680075BB1F023C40
:103A6400A8023CA87E017F00E5BE1270CFE5BD2F01
:103A7400FF50010E8E598F5A74091270CF74E68E5E
:103A8400048F05FF1270BF8D6A900095E070067573
:103A94006F0F0232FC75BB15023CA8023CA89000D3
:103AA40095E07003023BF37E017F00E5BE1270CF08
:103AB400E5BD2FFF50010E8E598F5A740412003940
:103AC4008F69900095E0B401159000E9E08569F0F4
:103AD400A4FFAEF07407120039EF9008EAF09000EA
:103AE40095E0B402159000E9E08569F0A4FFAEF01A
:103AF4007407120039EF9008E9F0900095E0B403E0
:103B0400028003023BD69000D6E07052E569C3946C
:103B140019500FD2289000B5E09008EDF09008F20B
:103B2400E4F0E569D394644004A2284002802D9017
:103B340008F2E004F09008F2E0FE900128E0B506F7
:103B44000B9008EDE004F09008F2E4F09008EDE04A
:103B540064966006900128E07002C2288063900099
:103B6400B5E070349000E9E08569F0A4FFAEF0742C
:103B7400FF8E048F05FF1270BFED9008EDF0AE517B
:103B8400AF52741EBE0006D39F4002D228E561D313
:103B940094E54002C2288029E569C3940A500DAE19
:103BA40051AF52741EBE0004D39F50028002D2282B
:103BB400E561D394E54002C2289000B5E09008ED99
:103BC400F09008EDE0C39405500674059008EDF0FC
:103BD400C22D900095E0B40414E569C39419500211
:103BE400D22DE569D394324002C22DC228800375D8
:103BF40069009000ECE07006756F110232FC75BB31
:103C040014023CA8023CA89000ECE07003023C952E
:103C14007E017F00E5BE1270CFE5BD2FFF50010E7F
:103C24008E598F5A90012CE075F010A4FDACF08CE5
:103C34005B8D5CEFD39DEE9C400912711A8E598FF7
:103C44005A8006755A00755900AE59AF5A740E124F
:103C540070CF9000F3E08E048F05FF1270BF8C5B71
:103C64008D5C74FFBC00039D5005756BFF8003855C
:103C74005C6BE56B75F00BA4FFAEF09000DAE08EA0
:103C8400048F05FF1270BF90089BECF0A3EDF08049
:103C940003756B00900090E0600575BB1A80037596
:043CA400BB188000C9
:103D0F000233050233080236410236440237CA0233
:103D1F0037CD0238B10238B402391902391C0239D1
:103D2F00C50239C8023A65023A68023A9F023AA2BE
:093D3F00023C08023C0B023CA806
:103CA800E56F75F00284AFF07E00EF4E7002D2EC43
:033CB800056F2273
:097100002582F58250020583226C
:0F008C0025E050020583258250020583F582226C
:10709E00EF2F500205832582F582E5833E2EF58380
:0170AE0022BF
:10711200CFC39FFF50011E22C3EF9DFFEE9CFE22B4
:087122000806B600021806225F
:0D70DD00A3E004F070061270F6E004F0224B
:0E003900048007C3CE13CECF13CFD5E0F6223E
:106FBD00BC000FBE0008ED8FF084FFADF022E4FEA3
:106FCD00FF22BE000DEF60FE54F0606F20E703025C
:106FDD007073EAC0E0EBC0E078017A0075F001EE65
:106FED0020E710EF25E0FFEE33FE0AC5F023C5F0D4
:106FFD0030E7F0EA5407F9096A7A007B006001086E
:10700D00C3EC9E40167004ED9F4010ED9FFDEC9E6D
:10701D00FCE5F0CA4ACA03F5F08005E5F003F5F08A
:10702D00C3EE13FEEF13FFD9D77908CACBCAD8D058
:10703D00EAFEEBFFD0E0FBD0E0FA22EC8FF084FC0F
:10704D00ED54F045F0C48FF084FEEDC454F045F0DE
:10705D00C48FF084FDEEC4FE54F02DFFEE540F3CB2
:10706D00FEADF07C0022790078008FF0EC7E0820D8
:10707D00E70DC3CD33CD33C933C9C833C8DEF08472
:10708D0049F9E5F08FF0BE00E6FD7C00E9FFE8FE72
:01709D0022D0
:0E70CF00F88FF0A4FFE5F0CE88F0A42EFE228C
:10000300EF8DF0A4F9A8F0EF8CF0A428F8EE8DF0B2
:06001300A428FEE9FF2213
:1070AF00600D782B0270B9007830D8FED5E0F82249
:1070BF00EEC0E07E00126FBDEFFDEEFCD0E0FE22D1
:0C70EA00EEC0E07E00126FBDD0E0FE2280
:03001B0002001EC2
:0300530002005652
:03009B00020071EF
:0300000002710981
:0971090075817575D000024C423D
:0B004800E5822FF582E5833EF5832260
:0A70F6000582D5820215831582225F
:10001E00C0E0C0F0C083C082C0D075D000124B6962
:0B002E00D0D0D082D083D0F0D0E032E0
:10005600C0E0C0F0C083C082C0D075D000124B6C27
:10006600D0D0D082D083D0F0D0E032C0E0C0F0C093
:1000760083C082C0D075D000124BA6D0D0D082D01B
:0600860083D0F0D0E0324F
:00000001FF
